:020000040000FA
:04000000ACEF00F071
:100008005582D9CF05F0DACF06F00F0112A91BD01F
:100018008EBC02D0839483928EA802D083A20ED085
:10002800899424EE04F0010EDBBE07D0000EDE5CDE
:10003800020EDE5802E3899201D089828EB883B21B
:1000480001D08984129912A17BD08EB883B289928B
:10005800901C086E8E1C076E04C409F005C40AF0D3
:100068000ABE03D0020E0A5C2FE28EA802D083A239
:100078002BD0094A0A2A09C004F40AC005F402C4AC
:1000880009F003C40AF0060E0924D96E040E0A20EA
:10009800DA6E08C0DFFF060E0924D96E060E0A20A4
:1000A800DA6E07C0DFFF094A0A2A0168010E026EEC
:1000B80009C003F00AC004F00150031602500416E8
:1000C80003C002F404C003F48EB883B2898489841F
:1000D8008EA0FED78EA802D083A202D0899401D028
:1000E800898424EE04F0010EDBBE07D0000EDE5C2E
:1000F800020EDE5802E3899201D0898207A81ED039
:100108000BD0838202D0838405D0839417D083A236
:1001180015D08394839212D00850016E026A02505F
:100128000DE10150040AF3E0100AF1E0340AE9E0B5
:100138001F0AF0E07F0AE7E01F0AE7E00F011291CB
:100148000E01CA9906C0DAFF05C0D9FF5592110001
:100158005BEF48F07CC0D9FF7DC0DAFFDE6ADD6A5C
:100168007EC00BF0BEEC43F00BC0B6F00CC0B7F08D
:100178000001B7BF0B0CD890B635D96EB735DA6E1B
:100188008C0ED926010EDA22DECFD0F0DDCFD1F0E9
:10019800D051D11101E10C0C7CC0D9FF7DC0DAFF30
:1001A800D0C0DEFFD1C0DDFFD0C0D9FFD1C0DAFF9B
:1001B800DF5012E020EE01F0D051D926D151DA22D9
:1001C800DF5011EC57F00001C26FC2B105D07F516A
:1001D800D8A4C2A5000C0A0CD0C0D9FFD1C0DAFF40
:1001E800DF6A20EE01F0D051D926D151DA22B6C00B
:1001F800DFFF20EE01F0D051D926D151DA22DF50AD
:1002080049EC3FF00001C26FC2B1030C7F5102E01C
:10021800C2B50A0CC96BCA6BCB6BCC6BD0C044F0AF
:10022800D1C045F0C9C046F0CAC047F0CBC048F0BD
:10023800CCC049F00EEC36F00001CF6FCF0501E0DD
:10024800D4D0CD6BCE6BCE5105E1040ECD5D01E36C
:1002580090D001D08ED0CDC080F0CEC081F0803B50
:10026800813BF00E811780510F0B8113F00E801720
:10027800D0C082F0D1C083F080518227815183237E
:10028800EC0E8225C36F010E8321C46F20EE04F0AB
:10029800C351D926C451DA22DF5005E1A86BA96BF6
:1002A800AA6BAB6B55D020EE09F0C351D926C451C7
:1002B800DA22DF50816F806B20EE0AF0C351D92615
:1002C800C451DA22DF50826F82C083F0846B856B61
:1002D800866B84C086F083C085F0846B836B20EEC8
:1002E8000BF0C351D926C451DA22DF50876F87C07B
:1002F80088F0896B8A6B8B6B88C08BF08A6B896BF3
:10030800886B835188118C6F845189118D6F855149
:100318008A118E6F86518B118F6F80518C11906F5F
:1003280081518D11916F000E8E11926F000E8F11F9
:10033800936F20EE08F0C351D926C451DA22DF505A
:100348009011A86F9151A96F9251AA6F9351AB6FF9
:10035800CD51040DF350980FD96EDA6AA8C0DEFFAC
:10036800A9C0DEFFAAC0DEFFABC0DEFFCD4BCE2B9F
:100378006AD7CD6BCE6BCD51CE1103E0CD07D8A097
:10038800CE07CD51040DF350980FD96EDA6ADECF3F
:10039800C9F0DECFCAF0DECFCBF0DECFCCF0C9514A
:1003A800CA11CB11CC1105E1000EAD6F020EAC6F76
:1003B80011D0D0C044F0D1C045F0C9C046F0CAC081
:1003C80047F0CBC048F0CCC049F00EEC36F0000145
:1003D800AC6FAD6BACC0CFF0CF5107E0CD4BCE2B9F
:1003E800CE5103E1040ECD5DCCE3030ECF1901E13C
:1003F800010CCF5101E00D0C20EE3AF0D051D92676
:10040800D151DA22DF50816F806B20EE39F0D05164
:10041800D926D151DA22DF508013020E81198011BA
:1004280001E00D0C20EE45F0D051D926D151DA2249
:10043800DF50816F806B20EE44F0D051D926D15126
:10044800DA22DF50801380C0C5F081C0C6F0C76BC8
:10045800C86BC551C611C711C81155E120EE53F03C
:10046800D051D926D151DA22DF50816F806B20EE2E
:1004780054F0D051D926D151DA22DF50826F82C090
:1004880083F0846B856B866B84C086F083C085F0AF
:10049800846B836B20EE55F0D051D926D151DA22E6
:1004A800DF50876F87C088F0896B8A6B8B6B88C039
:1004B8008BF08A6B896B886B835188118C6F8451A0
:1004C80089118D6F85518A118E6F86518B118F6FAF
:1004D80080518C11906F81518D11916F000E8E118A
:1004E800926F000E8F11936F20EE52F0D051D926E3
:1004F800D151DA22DF509011C56F9151C66F9251D8
:10050800C76F9351C86F20EE16F0D051D926D1513C
:10051800DA22C5C0DEFFC6C0DEFFC7C0DEFFC8C026
:10052800DEFF20EE3EF0D051D926D151DA2210EE6E
:1005380003F0D051E126D151E222DFCFE7FF20EED0
:1005480003F0D051D926D151DA22DE040AE020EE98
:1005580003F0D051D926D151DA22020EDE1801E07B
:100568000D0CC5C00BF0C6C00CF0C7C00DF0C8C05C
:100578000EF020EE03F0D051D926D151DA22DF5007
:100588000F6E106A116A126A37EC4EF00BC0C5F094
:100598000CC0C6F00DC0C7F00EC0C8F020EE3BF08E
:1005A800D051D926D151DA2210EE02F0D051E126ED
:1005B800D151E222DFCFE7FF20EE02F0D051D92659
:1005C800D151DA22DF50D8B40D0C20EE02F0D05110
:1005D800D926D151DA22DF50806F20EE02F0D051B7
:1005E800D926D151DA22DF50816F8105801501E0CB
:1005F8000D0C20EE40F0D051D926D151DA22DF502F
:10060800816F806B20EE3FF0D051D926D151DA228C
:10061800DF50801320EE08F0D051D926D151DA22CC
:1006280080C0DEFF81C0DDFF20EE08F0D051D92662
:10063800D151DA22DF50806F0F0E801701E00D0CC8
:1006480020EE42F0D051D926D151DA22DF50816F05
:10065800806B20EE41F0D051D926D151DA22DF50FB
:10066800801380C0BAF081C0BBF0BC6BBD6BBA51BF
:10067800BB11BC11BD1155E120EE4FF0D051D92668
:10068800D151DA22DF50816F806B20EE50F0D051CB
:10069800D926D151DA22DF50826F82C083F0846B71
:1006A800856B866B84C086F083C085F0846B836B12
:1006B80020EE51F0D051D926D151DA22DF50876F80
:1006C80087C088F0896B8A6B8B6B88C08BF08A6BCC
:1006D800896B886B835188118C6F845189118D6F58
:1006E80085518A118E6F86518B118F6F80518C11B5
:1006F800906F81518D11916F000E8E11926F000EC7
:100708008F11936F20EE4EF0D051D926D151DA22B5
:10071800DF509011BA6F9151BB6F9251BC6F9351DA
:10072800BD6F20EE3CF0D051D926D151DA22DF50EE
:10073800806F20EE3DF0D051D926D151DA22DF501A
:10074800816F8051B86F81C0B9F0B851B91101E11A
:100758000D0C20EE08F0D051D926D151DA22DECF87
:1007680080F0DDCF81F0040E826FD8908133803322
:10077800822FFBD7B8518025836FB9518121846FAF
:10078800856BD8B0852B866BC5518325B26FC65152
:100798008421B36FC7518521B46FC8518621B56FC5
:1007A800B251BA5DB351BB59B451BC59B551BD59D9
:1007B80001E20D0CB251BA5D0B6EB351BB590C6E10
:1007C800B451BC590D6EB551BD590E6E20EE02F0F4
:1007D800D051D926D151DA22DF500F6E106A116A32
:1007E800126AF9EC4EF00BC0BEF00CC0BFF00DC0A1
:1007F800C0F00EC0C1F00001BE51BF11C011C1113F
:1008080001E10D0C010ECF6FC151C01105E1F60ECB
:10081800BE5D0F0EBF5902E3020ECF6FC151C0116A
:1008280005E1F60EBE5DFF0EBF5902E3030ECF6F62
:10083800020EBE25806F000EBF21816F000EC02101
:10084800826F000EC121836F20EE12F0D051D9269D
:10085800D151DA2280C0DEFF81C0DEFF82C0DEFF18
:1008680083C0DEFF20EE1AF0D051D926D151DA220A
:10087800C9C0DEFFCAC0DEFFCBC0DEFFCCC0DEFFD2
:10088800B851C925806FB951CA21816F000ECB219B
:10089800826F000ECC21836F20EE1EF0D051D92636
:1008A800D151DA2280C0DEFF81C0DEFF82C0DEFFC8
:1008B80083C0DEFFB251C925806FB351CA21816F51
:1008C800B451CB21826FB551CC21836F20EE26F035
:1008D800D051D926D151DA2280C0DEFF81C0DEFF97
:1008E80082C0DEFF83C0DEFF030ECF1901E08CD08B
:1008F80020EE08F0D051D926D151DA22DE50DE1090
:1009080001E00D0C20EE5BF0D051D926D151DA224E
:10091800DF50816F806B20EE5CF0D051D926D15129
:10092800DA22DF50826F82C083F0846B856B866B1E
:1009380084C086F083C085F0846B836B20EE5DF005
:10094800D051D926D151DA22DF50876F87C088F07D
:10095800896B8A6B8B6B88C08BF08A6B896B886B11
:10096800835188118C6F845189118D6F85518A113B
:100978008E6F86518B118F6F80518C11906F8151C2
:100988008D11916F000E8E11926F000E8F11936F63
:1009980020EE5AF0D051D926D151DA22DF509011E9
:1009A800946F9151956F9251966F9351976F20EE76
:1009B80022F0D051D926D151DA2294C0DEFF95C059
:1009C800DEFF96C0DEFF97C0DEFF20EE12F0D051AA
:1009D800D926D151DA22DECF80F0DECF81F0DECF0A
:1009E80082F0DECF83F0020ED890803781378237CD
:1009F8008337E82EF9D780C0AEF081C0AFF082C04F
:100A0800B0F083C0B1F0B7D020EE08F0D051D926AD
:100A1800D151DA22DE50DE1001E10D0C20EE1EF07D
:100A2800D051D926D151DA22DECF80F0DECF81F045
:100A3800DECF82F0DECF83F0C5518025846FC651AA
:100A48008121856FC7518221866FC8518321876FA5
:100A580020EE22F0D051D926D151DA2284C0DEFF0F
:100A680085C0DEFF86C0DEFF87C0DEFF020ECF191D
:100A78006BE020EE12F0D051D926D151DA22DECF28
:100A880080F0DECF81F0DECF82F0DECF83F0010E82
:100A98008015846F856B866B876B20EE12F0D051C2
:100AA800D926D151DA22DECF88F0DECF89F0DECF29
:100AB8008AF0DECF8BF0030E8803F3CF8CF0F4CFEF
:100AC8008DF08E6B8F6B8903F3508D27F4508E2336
:100AD800000E8F238803F3508D27F4508E23000EC9
:100AE8008F23030E8A03F3508E27F4508F23000EB2
:100AF8008903F3508E27F4508F23000E8803F35098
:100B08008E27F4508F23030E8B03F3508F27000E8C
:100B18008A03F3508F27000E8903F3508F27000EA6
:100B28008803F3508F27D8908F338E338D338C33CF
:100B380084518C25AE6F85518D21AF6F86518E21E2
:100B4800B06F87518F2116D020EE12F0D051D926E0
:100B5800D151DA22DECF80F0DECF81F0DECF82F015
:100B6800DECF83F0D8908035AE6F8135AF6F823598
:100B7800B06F8335B16FFF0EAE25806F010EAF21C8
:100B8800816F000EB021826F000EB121836F0A0EB3
:100B980005D0D8908333823381338033E82EF9D758
:100BA80020EE16F0D051D926D151DA228051DE5CE0
:100BB8008151DE588251DE588351DE5801E20D0C16
:100BC80020EE0EF0D051D926D151DA22DE68DE6847
:100BD800DE68DD68DD52DD5210EE0AF0D051E12604
:100BE800D151E222DECFE6FFDECFE6FFDECFE6FF21
:100BF800DECFE6FF20EE05F0D051D926D151DA221A
:100C0800800EDF6E030ECF1901E0D3D120EE5FF026
:100C1800D051D926D151DA22DF50816F806B20EE76
:100C28005EF0D051D926D151DA22DF5080138005E9
:100C3800811101E0BED1D0C039F0D1C03AF0C92944
:100C48003B6E000ECA213C6E000ECB213D6E000E9D
:100C5800CC213E6EF5EC4BF0000901E0AAD1000171
:100C680020EE05F0D051D926D151DA22DF6A22EEE2
:100C78002DF0D051D926D151DA22DF50816F806B07
:100C880022EE2CF0D051D926D151DA22DF50801330
:100C9800550E801903E1AA0E8119D8A48AD120EE35
:100CA8002FF0D051D926D151DA22DF50816F806BD5
:100CB80020EE30F0D051D926D151DA22DF50826FA0
:100CC80082C083F0846B856B866B84C086F083C09A
:100CD80085F0846B836B20EE31F0D051D926D15149
:100CE800DA22DF50876F87C088F0896B8A6B8B6B3D
:100CF80088C08BF08A6B896B886B835188118C6FE5
:100D0800845189118D6F85518A118E6F86518B118F
:100D18008F6F80518C11906F81518D11916F000EE2
:100D28008E11926F000E8F11936F20EE2EF0D0511E
:100D3800D926D151DA22DF509011946F9151956FD5
:100D48009251966F9351976F520E941909E1520E72
:100D5800951906E1610E961903E1410E9719D8A479
:100D680028D122EE13F0D051D926D151DA22DF5002
:100D7800816F806B22EE14F0D051D926D151DA223E
:100D8800DF50826F82C083F0846B856B866B84C072
:100D980086F083C085F0846B836B22EE15F0D0510A
:100DA800D926D151DA22DF50876F87C088F0896B46
:100DB8008A6B8B6B88C08BF08A6B896B886B8351CD
:100DC80088118C6F845189118D6F85518A118E6FAE
:100DD80086518B118F6F80518C11906F81518D11BD
:100DE800916F000E8E11926F000E8F11936F22EE8D
:100DF80012F0D051D926D151DA22DF509011946FD8
:100E08009151956F9251966F9351976F720E9419F5
:100E180009E1720E951906E1410E961903E1610E7A
:100E28009719D8A4C6D022EE17F0D051D926D1519F
:100E3800DA22DF50816F806B22EE18F0D051D9266C
:100E4800D151DA22DF50826F82C083F0846B856BC8
:100E5800866B84C086F083C085F0846B836B22EE3A
:100E680019F0D051D926D151DA22DF50876F87C0C7
:100E780088F0896B8A6B8B6B88C08BF08A6B896B67
:100E8800886B835188118C6F845189118D6F8551BE
:100E98008A118E6F86518B118F6F80518C11906FD4
:100EA80081518D11916F000E8E11926F000E8F116E
:100EB800936F22EE16F0D051D926D151DA22DF50A5
:100EC8009011946F9151956F9251966F9351976FBE
:100ED80020EE0EF0D051D926D151DA2294C0DEFF8F
:100EE80095C0DEFF96C0DEFF97C0DEFF22EE1BF046
:100EF800D051D926D151DA22DF50816F806B22EE92
:100F08001CF0D051D926D151DA22DF50826F82C02D
:100F180083F0846B856B866B84C086F083C085F014
:100F2800846B836B22EE1DF0D051D926D151DA2281
:100F3800DF50876F87C088F0896B8A6B8B6B88C09E
:100F48008BF08A6B896B886B835188118C6F845105
:100F580089118D6F85518A118E6F86518B118F6F14
:100F680080518C11906F81518D11916F000E8E11EF
:100F7800926F000E8F11936F22EE1AF0D051D9267E
:100F8800D151DA22DF509011946F9151956F92519F
:100F9800966F9351976F20EE0AF0D051D926D15110
:100FA800DA2294C0DEFF95C0DEFF96C0DEFF97C050
:100FB800DEFFD0C0D9FFD1C0DAFFCFC0DFFF01010B
:100FC8008A4B8B2B000120EE06F0D051D926D15147
:100FD800DA228AC1DEFF8BC1DDFF000C0C6A0B6AC6
:100FE800BEEC56F00F0B0101F96F9A6B070E8C6E71
:100FF800010EFB6F9F6B0F0E0F01596F116B196B71
:10100800216B266B2E6B886889688A688A8E88901F
:1010180088928382020E0101FA6F78EC55F0889469
:101028008384889C839C889E838E8B688968700ED5
:101038000001606FFB0E616FA30E626FFF0E636F9E
:10104800FB0E646FFE0E656F310E666FFF0E676FE5
:10105800E0EC56F08A98858847EC55F017D0BB0E1F
:101068000001606FFE0E616F8FCF62F0636BE0EC82
:1010780056F0290E0001FC6F960EFB6F7F0EE82ECE
:10108800FED7FB2FFCD7FC2FFAD704008FB2E7D787
:10109800DEEC44F00101F96F890E0001606FFC0E6F
:1010A800616FF9C162F0636BE0EC56F00400520E18
:1010B8000001FC6F2B0EFB6F000EE82EFED7FB2FF6
:1010C800FCD7FC2FFAD700F0D250F00B0109D26EF2
:1010D800D09E0E01C691CF0ECF16CF82CF80C28987
:1010E8000F01138113891489F28E0E01BA89DFEC7E
:1010F8004FF08392839476EC47F076EC47F0000E3D
:101108000B6E340E90EC52F04C0E0F6EFF0E106EFC
:10111800BCEC4EF0A30E0F6EFF0E106EBCEC4EF042
:10112800000E0B6E390E90EC52F083800400DEEC5A
:1011380029F0EDC193FF1AEC39F034EC4FF0000EB2
:101148000B6E800E90EC52F02BEC56F0000E0B6EEE
:10115800800E90EC52F00101F9510F0D340EF3247A
:101168000F6E0C0EF420106EBCEC4EF0010199517C
:1011780001E1D4D0BE0E0001606FFD0E616FE0EC9E
:1011880056F016EC50F00FC0DFF110C0E0F111C0BE
:10119800E1F112C0E2F10101DF51E011E111E211C8
:1011A80017E1E60E0001606FFC0E616FDFC162F0AF
:1011B800E0C163F0E1C164F0E2C165F0E0EC56F033
:1011C8000A0E0E6E000E0F6A106A116A15EC52F0C4
:1011D8000101E36BE46BE4BF05D0E45119E1040EAF
:1011E800E35D16E2DC0E0001606FFF0E616FDF0E3B
:1011F8000101E325D96E010EE421DA6EDF5000010A
:10120800626F636BE0EC56F00101E34BE42BE3D72C
:101218009E0E0001606FFB0E616FE0EC56F03E0E13
:101228000001606FFC0E616FE0EC56F022EE00F0FA
:1012380000EECDF01F0EDBCFEBFFE806FCE2D00E90
:101248000001ED6FFF0EEE6FD0EC33F0CDC074F1FE
:10125800CEC075F1CFC076F1D0C077F101017451DD
:101268007511761177115AE0240E0001606FFC0E9B
:10127800616F74C162F075C163F076C164F077C1C3
:1012880065F0E0EC56F0000E0001A66F020EA76FA5
:1012980074C1FCF075C1FDF076C1FEF0FB6B000E69
:1012A800FB25A86F010EFC21A96F000EFD21AA6F76
:1012B800000EFE21AB6F14EC0FF0000E846F020ECF
:1012C800856F340E866F0A0E876F896B080E886FDC
:1012D800DD0E8A6F010E8B6FFEEC11F00101E56BDC
:1012E800E66BE6BF05D0E65119E1080EE55D16E2AA
:1012F800D80E0001606FFF0E616F340E0101E52505
:10130800D96E0A0EE621DA6EDF500001626F636B58
:10131800E0EC56F00101E54BE62BE3D79FAF12D086
:101328008A6883928382290E0001FC6F960EFB6FF8
:101338007F0EE82EFED7FB2FFCD7FC2FFAD707EC41
:101348003BF0EFD7FB5104E0020E9E6F2D0E0BD041
:10135800CE0E0001606FFD0E616FE0EC56F0010EDD
:1013680001019E6F040E9D6FD96BDA6BEA6B000E5C
:10137800E86F010EE76FE8BF05D0E85162E1040E9F
:10138800E75D5FE20F0EE703F3CFFBF0F4CFFCF06D
:10139800E803F3500001FC27240EFB250B6E0D0E0D
:1013A800FC210C6ED0EC53F00C5003E1030E0B5CE7
:1013B80044E32B0E0001606FFE0E616F0F0E0101FA
:1013C800E703F3CFFBF0F4CFFCF0E803F3500001A0
:1013D800FC27240EFB25626F0D0EFC21636FE0ECE9
:1013E80056F0E7C1FBF0E8C1FCF0050ED89000010B
:1013F800FB37FC37E82EFAD7000EFB25D26F020E1A
:10140800FC21D36F0F0E0101E703F3CFFDF0F4CFFA
:10141800FEF0E803F3500001FE27240EFD25D46FEB
:101428000D0EFE21D56F030ED66F48EC17F00101A3
:10143800DB6FDC6BDB513EEC52F00101E74BE82B34
:101448009AD79B0502E1070E8C6E020E9B1904E1E8
:101458000F01108B070E2D6F839E000E0B6EC00EB2
:1014680090EC52F02BEC56F0000E0B6EC00E90EC88
:1014780052F00101A1510CE0A10E0F6E010E106E89
:10148800BCEC4EF0380E0F6EFE0E106EBCEC4EF03B
:10149800910E0F6EFF0E106EBCEC4EF006D18EA8AA
:1014A800899478EC56F00B500C1001E1DFD0EAC1BA
:1014B800D8F1E90E0B6E010E0C6EAFEC4DF0010188
:1014C800EA6FE9B9EA9F350EEA1907E19E0E0001B5
:1014D800606FFB0E616FE0EC56F03A0E0001606F32
:1014E800FF0E616FEAC162F0636B0101010EE9A9A9
:1014F800000E0001646F656BE0EC56F00101E9A98C
:101508001ED0600EEA191BE15F0ED81918E1FA83A4
:101518002AEE34F09EC1DFFF2AEE35F09DC1DFFFD1
:101528008384496A020E486E92EC32F0839401017A
:10153800FA93536A97EC56F00101EA6BB6D0FB5167
:101548004AE0E951100B0001A96F000EAA6F0101D2
:10155800EA51DEEC3CF0A9C0EBF1AAC0ECF1080EB0
:101568000101EB19EC1101E100F0070E0101EB1983
:10157800EC1102E1DCEC50F0EB05EC1102E157EC68
:101588004AF0020EEB19EC1102E113EC3AF0030EEB
:10159800EB19EC1106E11AEC2DF0E4C0D9F1E5C025
:1015A800DAF1050E0101EB19EC1106E11EEC38F039
:1015B800EDC0D9F1EEC0DAF1090E0101EB19EC1119
:1015C80002E1FAEC49F00A0E0101EB19EC116DE1A8
:1015D80017EC57F06AD0E951100B486E000E496EAF
:1015E800EA513EEC22F048C0EBF149C0ECF1070E9D
:1015F8000101EB19EC1102E14AEC50F0020EEB1973
:10160800EC1102E1B8EC52F0EB05EC1102E165ECEB
:1016180041F0030EEB19EC1102E104EC53F0040E57
:10162800EB19EC1102E18FEC55F0050EEB19EC11FA
:1016380002E150EC44F0060E0101EB19EC1102E155
:101648001FEC57F0080EEB19EC1102E1BAEC3DF073
:10165800090EEB19EC1102E1F8EC46F00A0E010153
:10166800EB19EC1122E169EC45F01FD0DEEC44F0F7
:1016780001019A6F9B5119E0F9519A1916E0838E6E
:10168800000E0B6EC00E90EC52F02BEC56F0000ED4
:101698000B6EC00E90EC52F0070E0F6EFF0E106E20
:1016A800BCEC4EF09AC1F9F131D08FB22FD0050EB3
:1016B8000101D919DA112AE0F2D6BB0E0001606FD8
:1016C800FE0E616F8FCF62F0636BE0EC56F0290E6F
:1016D8000001FC6F960EFB6F7F0EE82EFED7FB2FE6
:1016E800FCD7FC2FFAD70400000E0B6EC00E90EC4E
:1016F80052F02BEC56F0000E0B6EC00E90EC52F030
:10170800540E0F6EFF0E106EBCEC4EF08FB2D5D794
:10171800090E0001FC6F1E0EFB6FE40EE82EFED7CB
:10172800FB2FFCD7FC2FFAD700F08394839200019B
:10173800D26BD36BA00ED46FFB0ED56FD66B43EC78
:101748004CF0F4D4A8C0BAF0A9C0BBF0AC51D96E23
:10175800DA6ADE6ADD6AA6C00CF0A7C00DF068EC94
:101768004DF00001B96FB95102E0B951120020EEF5
:1017780005F0A651D926A751DA22DF5008E020EE5D
:1017880005F0A651D926A751DA22DF50120020EE23
:1017980004F0A651D926A751DA22DFA2070C20EEC1
:1017A80006F0A651D926A751DA2210EE06F0A65166
:1017B800E126A751E222E6CFB1F0E6CFB2F0E6CFBC
:1017C800B3F0E6CFB4F0AA51B125B56FAB51B22151
:1017D800B66F000EB321B76F000EB421B86FDE509C
:1017E800B55DDE50B659DE50B759DE50B85901E341
:1017F800E1D2AA6BAB6BDED220EE06F0A651D92659
:10180800A751DA22FF0EDE14AD6F010EDE14AE6FA3
:10181800000EDE14AF6F000EDE14B06FAD51AE11C6
:10182800AF11B01101E032D220EE06F0A651D92650
:10183800A751DA22DECFADF0DECFAEF0DECFAFF0CB
:10184800DECFB0F00A0E05D0D890B033AF33AE3348
:10185800AD33E82EF9D7A6C0D9FFA7C0DAFF10EE3E
:1018680002F0DE50E126DD50E222E750B16FB1050B
:10187800AD15BC6FBC5101E099D020EE06F0A65121
:10188800D926A751DA22DE50DE10DE10DE1022E162
:1018980020EE0EF0A651D926A751DA22DECFC3F0EA
:1018A800DECFC4F0DECFC5F0DECFC6F0C351C41121
:1018B800C511C6112FE1A6C0D9FFA7C0DAFFDECF38
:1018C8008FF0DDCF90F0916B926B936B946BE9EC9A
:1018D8002FF018D0A6C0D9FFA7C0DAFFDECF8FF04F
:1018E800DDCF90F020EE12F0A651D926A751DA22CA
:1018F800DECF91F0DECF92F0DECF93F0DECF94F022
:10190800E9EC2FF08FC0C3F090C0C4F091C0C5F0CF
:1019180092C0C6F0C351C411C511C61101E14ED21F
:10192800C305C411C511C61109E120EE05F0A65181
:10193800D926A751DA22020EDF6E020CC3290FE165
:10194800C4290DE1C5290BE1C62909E120EE05F0FE
:10195800A651D926A751DA22010EDF6E010C20EE1E
:1019680012F0A651D926A751DA22C3C0DEFFC4C09F
:10197800DEFFC5C0DEFFC6C0DEFF20EE0EF0A651BA
:10198800D926A751DA22DE50DE10DE10DE100EE175
:1019980020EE0EF0A651D926A751DA22C3C0DEFFE9
:1019A800C4C0DEFFC5C0DEFFC6C0DEFF20EE16F0F5
:1019B800A651D926A751DA22A6C0E1FFA7C0E2FFA7
:1019C80000EE2AF0E650E926E550EA22DE50EE184D
:1019D80016E1DE50EE1813E1DE50EE1810E1DE508D
:1019E800EE180DE1A6C0D9FFA7C0DAFFDECF24F0BC
:1019F800DDCF25F0C2EC40F0000901E083D1A6C09C
:101A0800D9FFA7C0DAFFDECF0BF0DDCF0CF0000165
:101A180020EE12F0A651D926A751DA22DECF0DF01A
:101A2800DECF0EF0DECF0FF0DECF10F0F0EC45F099
:101A38000BC0BFF00CC0C0F00DC0C1F00EC0C2F0AA
:101A48000001BF51C011C111C21101E16ED7BC51D3
:101A5800BF27000EC023C123C223AAC0ADF0ABC06C
:101A6800AEF0090EAF6FD890AE33AD33AF2FFBD7C2
:101A7800ADC0BDF0AEC0BEF0BD51BE1101E1C3D0D6
:101A8800BC51BD25AD6F000EBE21AE6FA6C0D9FFFB
:101A9800A7C0DAFF10EE02F0DE50E126DD50E222A8
:101AA800E750AF6FB06BAD51AF5DAE51B05912E2B8
:101AB800A6C0D9FFA7C0DAFF10EE02F0DE50E1267B
:101AC800DD50E222E750AD6FBC51AD5DBD6FBE6B1E
:101AD800D8A0BE07BAC01AF0BBC01BF0BFC01CF02C
:101AE800C0C01DF0C1C01EF0C2C01FF0BDC020F0B4
:101AF800BEC021F0A6C0D9FFA7C0DAFF10EE01F0E2
:101B0800DE50E126DD50E222E750E9EC47F000091B
:101B180001E0F8D00001BD51AD6FBE51AE6FAF6BA3
:101B2800B06BA6C0D9FFA7C0DAFF10EE2AF0DE50CE
:101B3800E126DD50E222E6CFB1F0E6CFB2F0E6CF03
:101B4800B3F0E6CFB4F0BF51B15DB56FC051B25933
:101B5800B66FC151B359B76FC251B459B86FAD51CF
:101B6800B55DAE51B659AF51B759B051B8593CE20D
:101B7800A6C0D9FFA7C0DAFFDECFADF0DDCFAEF04B
:101B88002E0EAD250B6E000EAE210C6EA6C0D9FF31
:101B9800A7C0DAFF10EE2AF0DE50E126DD50E2227F
:101BA800E6CFAFF0E5CFB0F0BF51AF5FC051B05B4B
:101BB800090ED890AF37B037E82EFBD7AF51BA250A
:101BC8000D6EB051BB210E6E020E106E0F6A11EC35
:101BD80054F0A6C0D9FFA7C0DAFF10EE04F0DE501B
:101BE800E126DD50E222E76ABDC0ADF0BEC0AEF02E
:101BF800090ED890AD37AE37E82EFBD7ADC0C7F089
:101C0800AEC0C8F0BBD020EE0AF0A651D926A75125
:101C1800DA2210EE06F0A651E126A751E222DE50A4
:101C2800E65CDE50E658DE50E658DE50E6581FE324
:101C3800A6C0D9FFA7C0DAFFDECF24F0DDCF25F09C
:101C4800C2EC40F0000901E05DD0A6C0D9FFA7C0F2
:101C5800DAFF10EE2AF0DE50E126DD50E222BFC0A6
:101C6800E6FFC0C0E6FFC1C0E6FFC2C0E6FF000154
:101C780020EE16F0A651D926A751DA22BFC0DEFF02
:101C8800C0C0DEFFC1C0DEFFC2C0DEFFAD69010E0D
:101C9800AE6F20EE06F0A651D926A751DA22DECF84
:101CA800AFF0DDCFB0F0AD51AF17AE51B017AF51B7
:101CB8000008C76FB051D8A0E82A0208C86FC751FA
:101CC800AA5DC851AB5904E2AAC0C7F0ABC0C8F0BE
:101CD800A6C0D9FFA7C0DAFFDECF39F0DDCF3AF0D2
:101CE80020EE16F0A651D926A751DA22DECF3BF016
:101CF800DECF3CF0DECF3DF0DECF3EF0F5EC4BF032
:101D0800000902E0000122D60001AD69010EAE6FA4
:101D180020EE06F0A651D926A751DA22DECFAFF081
:101D2800DDCFB0F0AD51AF17AE51B017A6C0D9FF97
:101D3800A7C0DAFFDECFB1F0DDCFB2F0AF51B127E7
:101D4800B051B2232E0EB1250B6E000EB2210C6ECF
:101D5800BAC00DF0BBC00EF0C7C00FF0C8C010F07D
:101D680011EC54F0A6C0D9FFA7C0DAFF10EE04F0BA
:101D7800DE50E126DD50E222010EE76EC751BA2798
:101D8800C851BB2320EE06F0A651D926A751DA2266
:101D9800C751DE26C851DE22000EDE22DE22AC51FB
:101DA800D96EDA6AC751DE26C851DD22C751AA5F4B
:101DB800C851AB5BAA51AB1101E01ED520EE06F06D
:101DC800A651D926A751DA2210EE0AF0A651E1262B
:101DD800A751E222DE50E65CDE50E658DE50E658B7
:101DE800DE50E65814E220EE06F0A651D926A75197
:101DF800DA2210EE0AF0A651E126A751E222DECF40
:101E0800E6FFDECFE6FFDECFE6FFDECFE6FF20EE21
:101E180004F0A651D926A751DA22000EDB8A000C5D
:101E2800A6C00CF0A7C00DF068EC4DF00001C06F23
:101E3800C05102E0C051120020EE05F0A651D9268B
:101E4800A751DA22DF5008E020EE05F0A651D92686
:101E5800A751DA22DF50120020EE0AF0A651D92647
:101E6800A751DA22A851DE5CA951DE58AA51DE58E2
:101E7800AB51DE5816E220EE04F0A651D926A75140
:101E8800DA22DFB20ED020EE0AF0A651D926A751E9
:101E9800DA22DECFA8F0DECFA9F0DECFAAF0DECFBF
:101EA800ABF020EE06F0A651D926A751DA22DECFF4
:101EB800BCF0DECFBDF0DECFBEF0DECFBFF0C16B31
:101EC800C26BC36BC46B20EE06F0A651D926A7518E
:101ED800DA22C1C0DEFFC2C0DEFFC3C0DEFFC4C05D
:101EE800DEFFA851A911AA11AB1101E119D2A6C0B0
:101EF800D9FFA7C0DAFF10EE02F0DE50E126DD5070
:101F0800E222E750AC6FACC0ADF0AE6BAF6BB06B1C
:101F1800090ED890AD37AE37AF37B037E82EF9D7BE
:101F2800ADC0C5F0AEC0C6F0AFC0C7F0B0C0C8F015
:101F3800BC51BD11BE11BF1101E196D0FF0EA825FD
:101F48000B6EFF0EA9210C6EFF0EAA210D6EFF0E5F
:101F5800AB210E6EC5C00FF0C6C010F0C7C011F09F
:101F6800C8C012F0F9EC4EF00BC0ACF00CC0ADF0EC
:101F78000DC0AEF00EC0AFF0FF0E0001BC250B6E19
:101F8800FF0EBD210C6EFF0EBE210D6EFF0EBF2190
:101F98000E6EC5C00FF0C6C010F0C7C011F0C8C0A3
:101FA80012F0F9EC4EF00B500001AC5D0C50AD593D
:101FB8000D50AE590E50AF5957E3FF0EC525AC6F03
:101FC800FF0EC621AD6FFF0EC721AE6FFF0EC821F1
:101FD800AF6FAC1DB06FAD1DB16FAE1DB26FAF1D51
:101FE800B36FFF0EBC25B46FFF0EBD21B56FFF0E9A
:101FF800BE21B66FFF0EBF21B76FB051B415B86FD1
:10200800B151B515B96FB251B615BA6FB351B7150D
:10201800BB6F20EE06F0A651D926A751DA22B8C028
:10202800DEFFB9C0DEFFBAC0DEFFBBC0DEFF20EEB8
:1020380006F0A651D926A751DA22DE50A85FDE5055
:10204800A95BDE50AA5BDD50AB5B20EE12F0A65117
:10205800D926A751DA22DECFC9F0DECFCAF0DECF0B
:10206800CBF0DECFCCF064D020EE0EF0A651D9260E
:10207800A751DA22DECFC9F0DECFCAF0DECFCBF02F
:10208800DECFCCF0C951CA11CB11CC1143E1A6C0A7
:10209800D9FFA7C0DAFFDECF8FF0DDCF90F0916BCC
:1020A800926B936B946BE9EC2FF08FC0C9F090C0E2
:1020B800CAF091C0CBF092C0CCF0C905CA11CB11BF
:1020C800CC1109E120EE05F0A651D926A751DA2254
:1020D800020EDF6E020CC9290FE1CA290DE1CB29D6
:1020E8000BE1CC2909E120EE05F0A651D926A7512C
:1020F800DA22010EDF6E010C20EE0EF0A651D92671
:10210800A751DA22C9C0DEFFCAC0DEFFCBC0DEFF9E
:10211800CCC0DEFF20EE12F0A651D926A751DA2254
:10212800C9C0DEFFCAC0DEFFCBC0DEFFCCC0DEFF09
:10213800C951CA11CB11CC1101E095D0F1D020EED4
:1021480004F0A651D926A751DA22DFA228D0A6C0CA
:10215800D9FFA7C0DAFFDECF8FF0DDCF90F0C9C07E
:1021680091F0CAC092F0CBC093F0CCC094F0E9ECE7
:102178002FF08FC0C9F090C0CAF091C0CBF092C0C8
:10218800CCF0C951CA11CB11CC1123E1C5C0A8F0BC
:10219800C6C0A9F0C7C0AAF0C8C0ABF06ED0A6C030
:1021A800D9FFA7C0DAFFDECF44F0DDCF45F0C9C0C4
:1021B80046F0CAC047F0CBC048F0CCC049F008ECA4
:1021C8001CF044C0C9F045C0CAF046C0CBF047C0B7
:1021D800CCF00001C92907E1CA2905E1CB2903E1AF
:1021E800CC2901E180D7CC51CB11CA1104E1020EF0
:1021F800C95D01E267D7A6C0D9FFA7C0DAFF10EE14
:1022080012F0DE50E126DD50E222E650C95DE650CC
:10221800CA59E650CB59E650CC5901E353D720EEC2
:1022280012F0A651D926A751DA22C9C0DEFFCAC0CA
:10223800DEFFCBC0DEFFCCC0DEFF20EE06F0A651ED
:10224800D926A751DA22C551DE26C651DE22C7514A
:10225800DE22C851DE22C551A85FC651A95BC7510D
:10226800AA5BC851AB5BA851C55DA951C659AA5113
:10227800C759AB51C85901E262D720EE06F0A65102
:10228800D926A751DA22A851DE26A951DE22AA5161
:10229800DE22AB51DE22A851AC6F010EA915AD6F3D
:1022A800AE6BAF6BAC11AE11AF113AE0A6C0D9FF5F
:1022B800A7C0DAFFDECF0BF0DDCF0CF0C9C00DF000
:1022C800CAC00EF0CBC00FF0CCC010F0F0EC45F057
:1022D8000BC0C1F00CC0C2F00DC0C3F00EC0C4F0FA
:1022E8000001C151C211C311C41101E1EBD6A8C04C
:1022F800ACF0A9C0ADF0AAC0AEF0ABC0AFF00A0E0A
:1023080005D0D890AF33AE33AD33AC33E82EF9D720
:10231800AC51C127AD51C223AE51C323AF51C42321
:1023280020EE06F0A651D926A751DA22FF0EDE14B8
:10233800AC6F010EDE14AD6F000EDE14AE6F000E32
:10234800DE14AF6FAC51AD11AE11AF1120E020EE2D
:1023580016F0A651D926A751DA22C151DE1809E193
:10236800C251DE1806E1C351DE1803E1C451DE187C
:102378000EE020EE16F0A651D926A751DA22C1C0E8
:10238800DEFFC2C0DEFFC3C0DEFFC4C0DEFF20EE3A
:1023980006F0A651D926A751DA2210EE0AF0A65166
:1023A800E126A751E222DE50E65CDE50E658DE5018
:1023B800E658DE50E65801E33DD520EE06F0A6517A
:1023C800D926A751DA2210EE0AF0A651E126A75124
:1023D800E222DECFE6FFDECFE6FFDECFE6FFDECF8E
:1023E800E6FF20EE04F0A651D926A751DA22000E06
:1023F800DB8A20D586C0A1F087C0A2F08AC0D9FFA9
:102408008BC0DAFFDE6ADD6A84C00CF085C00DF08F
:1024180068EC4DF000019C6F9C5102E09C51120049
:1024280020EE05F08451D9268551DA22DF5008E0E4
:1024380020EE05F08451D9268551DA22DF501200AA
:1024480020EE04F08451D9268551DA22DFA0070C4A
:1024580020EE06F08451D9268551DA22DECF8CF0A1
:10246800DECF8DF0DECF8EF0DECF8FF020EE0AF0DB
:102478008451D9268551DA22DECF90F0DECF91F053
:10248800DECF92F0DECF93F08C51905D986F8D5136
:102498009159996F8E5192599A6F8F5193599B6F99
:1024A80088518C6F89518D6F8E6B8F6B8C51985DB5
:1024B8008D5199598E519A598F519B5901E34BD29D
:1024C80098C088F099C089F046D220EE06F0845171
:1024D800D9268551DA22FF0EDE148C6F010EDE1428
:1024E8008D6F000EDE148E6F000EDE148F6F8C5110
:1024F8008D118E118F1101E0A5D120EE06F08451C7
:10250800D9268551DA22DECF8CF0DECF8DF0DECFF2
:102518008EF0DECF8FF00A0E05D0D8908F338E3331
:102528008D338C33E82EF9D784C0D9FF85C0DAFF04
:1025380010EE02F0DE50E126DD50E222E750906F07
:1025480090058C15A36FA3516AE120EE06F0845123
:10255800D9268551DA22DE50DE10DE10DE100FE1BA
:1025680020EE0EF08451D9268551DA22DECF9DF077
:10257800DECF9EF0DECF9FF0DECFA0F020D084C06B
:10258800D9FF85C0DAFFDECF44F0DDCF45F020EE7D
:1025980012F08451D9268551DA22DECF46F0DECFFB
:1025A80047F0DECF48F0DECF49F008EC1CF044C01D
:1025B8009DF045C09EF046C09FF047C0A0F00001C6
:1025C800A0519F119E110CE1020E9D5D09E220EEC3
:1025D80005F08451D9268551DA22020EDF6E020CED
:1025E8009D290FE19E290DE19F290BE1A02909E111
:1025F80020EE05F08451D9268551DA22010EDF6ECE
:10260800010C20EE12F08451D9268551DA229DC0A2
:10261800DEFF9EC0DEFF9FC0DEFFA0C0DEFF84C0DD
:10262800D9FF85C0DAFFDECF0BF0DDCF0CF020EE4E
:1026380012F08451D9268551DA22DECF0DF0DECF93
:102648000EF0DECF0FF0DECF10F0F0EC45F00BC04F
:10265800A4F00CC0A5F00DC0A6F00EC0A7F00001B4
:10266800A451A511A611A71101E1B1D7A351A4271F
:10267800000EA523A623A72388C08CF089C08DF05F
:10268800090E8E6FD8908D338C338E2FFBD78CC06C
:10269800A8F08DC0A9F0A851A91101E1C5D0A35196
:1026A800A8258C6F000EA9218D6F84C0D9FF85C025
:1026B800DAFF10EE02F0DE50E126DD50E222E750AC
:1026C8008E6F8F6B8C518E5D8D518F5912E284C045
:1026D800D9FF85C0DAFF10EE02F0DE50E126DD50AA
:1026E800E222E7508C6FA3518C5DA86FA96BD8A02C
:1026F800A907A1C01AF0A2C01BF0A4C01CF0A5C075
:102708001DF0A6C01EF0A7C01FF0A8C020F0A9C0E9
:1027180021F084C0D9FF85C0DAFF10EE01F0DE5049
:10272800E126DD50E222E75007EC4BF0000901E01A
:10273800C5D084C0D9FF85C0DAFF10EE04F0DE50A2
:10274800E126DD50E222E7505FE00001A8518C6FDE
:10275800A9518D6F8E6B8F6B84C0D9FF85C0DAFF4E
:1027680010EE2AF0DE50E126DD50E222E6CF90F0AE
:10277800E6CF91F0E6CF92F0E6CF93F0A451905DCA
:10278800946FA5519159956FA6519259966FA7517B
:102798009359976F8C51945D8D5195598E519659D7
:1027A8008F51975931E284C0D9FF85C0DAFF10EE06
:1027B8002AF0DE50E126DD50E222E6CF8CF0E5CFAC
:1027C8008DF0A4518C5FA5518D5B090ED8908C3784
:1027D8008D37E82EFBD78C51A1250B6E8D51A22188
:1027E8000C6E84C0D9FF85C0DAFFDECF8EF0DDCF56
:1027F8008FF02E0E8E250D6E000E8F210E6E020E9E
:10280800106E0F6A11EC54F0A8C08CF0A9C08DF0BE
:10281800090ED89000018C378D37E82EFAD78CC076
:10282800AAF08DC0ABF07AD020EE16F08451D926EC
:102838008551DA22A4C0DEFFA5C0DEFFA6C0DEFFF8
:10284800A7C0DEFF8C69010E8D6F20EE06F0845163
:10285800D9268551DA22DECF8EF0DDCF8FF08C516C
:102868008E178D518F178E510008AA6F8F51D8A0DF
:10287800E82A0208AB6FAA51885DAB51895904E276
:1028880088C0AAF089C0ABF084C0D9FF85C0DAFF40
:10289800DECF39F0DDCF3AF020EE16F08451D9269C
:1028A8008551DA22DECF3BF0DECF3CF0DECF3DF0C3
:1028B800DECF3EF0F5EC4BF0000902E0000198D6BF
:1028C800A1C00BF0A2C00CF000018C69010E8D6F45
:1028D80020EE06F08451D9268551DA22DECF8EF01B
:1028E800DDCF8FF08C518E178D518F1784C0D9FF93
:1028F80085C0DAFFDECF90F0DDCF91F08E519027C2
:102908008F5191232E0E90250D6E000E91210E6E83
:10291800AAC00FF0ABC010F011EC54F0AA51A127D7
:10292800AB51A22320EE06F08451D9268551DA2234
:10293800AA51DE26AB51DE22000EDE22DE228AC03C
:10294800D9FF8BC0DAFFAA51DE26AB51DD22AA518E
:10295800885FAB51895B8851891101E0B6D5000CBD
:10296800276E266A1FD2275009E14F5007E0266AD2
:102978000101896B0A0E8BD0839084D2020E27182E
:1029880007E14F5005E0266A0101896B140E7FD0DC
:102998001F0E27642FD0300E27602CD04F502AE00E
:1029A8002750E00F506E266A5050200D0A0EF3246F
:1029B800D96E020EF420DA6EDE50DE10DE10DE1064
:1029C80003E0030E50642BD0010E4E6E5050140DD0
:1029D800130EF324D96E010EF420DA6E5050140D44
:1029E800130EF324E16E010EF420E26EE7500409A1
:1029F800DF6E15D03F0E276416D0500E276013D017
:102A08004F5011E05050140D000EF324D96E010EF2
:102A1800F420DA6E2750C00FDF6E266A4E6A010175
:102A2800886B896BA9D7310E271807E14F5005E04D
:102A38000C0E0101896F1D0EACD1340E271807E169
:102A48004F5005E00101886B896B266A95D7350ED2
:102A5800271808E14F5006E0266A0D0E0101896F1C
:102A6800AC0E15D0370E271808E14F5006E08380CA
:102A78000E0E0101896F750E8CD10D0E271809E114
:102A88004F5007E0266A020E0101896FBC0E886F5D
:102A980073D7100E271807E14F5005E0030E010108
:102AA800896FE90E76D1180E271807E14F5005E017
:102AB800070E0101896F090E6CD13B0E271807E13B
:102AC8004F5005E00E0E0101896F7E0E62D13E0E59
:102AD800271801E0D7D14F5001E1D4D10F0E0101E1
:102AE800896F3D0E56D15050140D010EF324D96E46
:102AF800010EF420DA6E27C0DFFF030E0101896F93
:102B0800EA0E47D15050140D020EF324D96E010E6F
:102B1800F420DA6E27C0DFFF030E0101896FEB0E88
:102B280038D15050140D030EF324D96E010EF42041
:102B3800DA6E27C0DFFF030E0101896FEC0E29D181
:102B48005050140D040EF324D96E010EF420DA6EE1
:102B580027C0DFFF030E0101896FED0E1AD1505017
:102B6800140D050EF324D96E010EF420DA6E27C079
:102B7800DFFF030E0101896FEE0E0BD15050140DCB
:102B8800060EF324D96E010EF420DA6E27C0DFFF9B
:102B98005050140D060EF324D96E010EF420DA6E8F
:102BA800DF500B6E0BC00CF00D6A0E6A0F6A0EC078
:102BB8000FF00DC00EF00CC00DF00C6A5050140D43
:102BC800050EF324D96E010EF420DA6EDF50106E74
:102BD80010C011F0126A136A146A12C014F011C0FE
:102BE80013F0126A116A5050140D040EF324D96EB2
:102BF800010EF420DA6EDF50156E15C016F0176A54
:102C0800186A196A16C019F0186A176A166A5050B5
:102C1800140D030EF324D96E010EF420DA6EDF5082
:102C280016241A6E000E17201B6E000E18201C6E3C
:102C3800000E19201D6E11501A241E6E12501B20F2
:102C48001F6E13501C20206E14501D20216E0C5036
:102C58001E24226E0D501F20236E0E502020246E3D
:102C68000F502120256E5050140D070EF324D96EF5
:102C7800010EF420DA6E22C0DEFF23C0DEFF24C07E
:102C8800DEFF25C0DEFF70D05050140D120EF32465
:102C9800D96E010EF420DA6E27C0DFFF070E01019E
:102CA800896F0A0E76D05050140D110EF324D96E88
:102CB800010EF420DA6E27C0DFFF070E0101896FCD
:102CC8000B0E67D05050140D100EF324D96E010E60
:102CD800F420DA6E27C0DFFF070E0101896F0C0EA2
:102CE80058D05050140D0F0EF324D96E010EF42055
:102CF800DA6E27C0DFFF38D00101886B896B4E6A16
:102D08003BD627C06CF10F0E0101896F3E0E41D0F2
:102D180027C06DF10F0E0101896F3F0E3AD027C011
:102D28006EF10F0E0101896F400E33D027C06FF18D
:102D38000F0E0101896F410E2CD027C070F10F0EC4
:102D48000101896F420E25D027C071F10F0E0101D4
:102D5800896F430E1ED027C072F10F0E0101896FD3
:102D6800440E17D027C073F10101886B896B8AD094
:102D78000C0E0101896F1E0E0CD00C0E0101896F1B
:102D88001C0E886F0A0E266EF7D50E0E0101896F8C
:102D9800760E886F77D00101886B896B090E266ED5
:102DA800838070D088C10BF089C10CF00C5011E001
:102DB800030A13E0040A25E00B0A31E0010A35E0B2
:102DC800030A38E0010A3FE0130A57E03B0A58E0DB
:102DD80059D00B5001E1C7D555D00B50E90A01E194
:102DE80082D6030A01E18ED6010A01E19AD6070AC2
:102DF80001E1A6D6010A01E1B2D6030A01E1BED675
:102E080041D00B50090A01E13FD7030A01E14BD732
:102E1800010A01E157D7070A01E163D733D00B5004
:102E28001D0AA6E0030AA9E02DD00B50480A9CE031
:102E3800E40A28D00B50750AA8E0030AACE0080A97
:102E480001E15AD71FD00B503D0A01E15AD7030AB6
:102E580001E15ED7010A01E162D77F0A01E166D785
:102E6800010A01E16AD7030A01E16ED7010A01E10B
:102E780072D7070A01E176D705D00B502A0A02D08B
:102E88000B500F0A26501200D251D31101E1090C40
:102E9800D2C0D9FFD3C0DAFFDE6ADD6A8CC1C2F1C5
:102EA8008DC1C3F11F0ED617C20E7C6F010E7D6F48
:102EB800D40E7E6FD651FE0B7F6FAEEC00F0010191
:102EC800BF6FBF5101E040D2AB0ED66F010ED76F76
:102ED800C20E0001BF6F010EC06FD4C0C1F0D5C0D3
:102EE800C2F007EC40F00101BF6FD4C1C0F1D5C1F9
:102EF800C1F1BF5105E1C051C11102E1060EBF6F1A
:102F0800D6C0D7F01C0E0001D71701E114D101017A
:102F1800BF5113E0040EBF1909E1C20E0001C36FCF
:102F2800010EC46F99EC49F00101BF6F0001D6870B
:102F3800D4C1C0F1D5C1C1F113D020EE0BF0C051FE
:102F4800D926C151DA22DF500001D76F110ED717E9
:102F580002E0070E03D0D6A503D0080E0101BF6F0B
:102F68000101BF5101E002D10001D6A7FFD0010144
:102F7800BB6BBC6B210EBD6F460EBE6F20EE0EF014
:102F8800C051D926C151DA22DF6A20EE0FF0C051B4
:102F9800D926C151DA22BCC1DFFF20EE10F0C051A2
:102FA800D926C151DA22BDC1DFFF20EE11F0C05190
:102FB800D926C151DA22BEC1DFFF20EE16F0C0517A
:102FC800D926C151DA22DF6A20EE17F0C051D9267E
:102FD800C151DA22BCC1DFFF20EE18F0C051D9265A
:102FE800C151DA22BDC1DFFF20EE19F0C051D92648
:102FF800C151DA22BEC1DFFF20EE0BF0C051D92645
:10300800C151DA22DF6A20EE1CF0C051D926C15125
:10301800DA22DF6A20EE1DF0C051D926C151DA222A
:10302800DF6A20EE1EF0C051D926C151DA22DF6ACC
:1030380020EE1FF0C051D926C151DA22DF6AC2C181
:103048000BF0C3C10CF0C0C10DF0C1C10EF0B2EC61
:103058004AF00BC0B7F10CC0B8F10DC0B9F10EC001
:10306800BAF1C0C10BF0C1C10CF00D6A0E6A0F6A4B
:10307800106AAFEC53F0010120EE04F0C251D926DA
:10308800C351DA22010EDF6EB751B811B911BA1166
:103098006DE020EE2AF0C251D926C351DA22DECFE4
:1030A800BBF1DECFBCF1DECFBDF1DECFBEF1C2C1D8
:1030B8008FF0C3C190F0B7C191F0B8C192F0B9C117
:1030C80093F0BAC194F028EC43F00101BF6FBF51EF
:1030D8004DE1FF0EB7250001D76FFF0E0101B821A2
:1030E8000001D86FFF0E0101B9210001D96FFF0E51
:1030F8000101BA210001DA6F010120EE0AF0C25184
:10310800D926C351DA22D7C0DEFFD8C0DEFFD9C026
:10311800DEFFDAC0DEFFC2C139F0C3C13AF0BBC17D
:103128003BF0BCC13CF0BDC13DF0BEC13EF0F5EC8A
:103138004BF001011AD00101BF5118E120EE0BF04C
:10314800C051D926C151DA22DFA802D0040E0DD011
:103158000001D6A30BD0010120EE0BF0C051D926F7
:10316800C151DA22DFA002D0070EBF6F0101BF51A3
:1031780023E10001D6B7D68B010120EE2AF0C25117
:10318800D926C351DA22000110EE1AF0D251E126F5
:10319800D351E222DECFE6FFDECFE6FFDECFE6FF49
:1031A800DECFE6FF20EE1EF0D251D926D351DA2227
:1031B800C0C1DEFFC1C1DDFF0101BF5101E0C4D0C4
:1031C800000120EE04F0D251D926D351DA22D6C01C
:1031D800DFFF20EE05F0D251D926D351DA22DF6A7B
:1031E800C2C10BF0C3C10CF0C0C10DF0C1C10EF0DB
:1031F800B2EC4AF0000120EE0EF0D251D926D3519C
:10320800DA220BC0DEFF0CC0DEFF0DC0DEFF0EC0F1
:10321800DEFF010120EE1DF0C051D926C151DA228E
:10322800DF500001D86FD76B010120EE1EF0C051AE
:10323800D926C151DA22DF500001D96FD9C0DAF09E
:10324800DB6BDC6BDD6BDBC0DDF0DAC0DCF0DB6B8D
:10325800DA6B010120EE1FF0C051D926C151DA22E4
:10326800DF500001DE6FDEC0DFF0E06BE16BE26B88
:10327800DFC0E2F0E16BE06BDF6BDA51DF11E36F87
:10328800DB51E011E46FDC51E111E56FDD51E21132
:10329800E66FD751E311E76FD851E411E86F000EDC
:1032A800E511E96F000EE611EA6F010120EE1CF04E
:1032B800C051D926C151DA22DF500001E711EB6F66
:1032C800E851EC6FE951ED6FEA51EE6F20EE0AF02C
:1032D800D251D926D351DA22EBC0DEFFECC0DEFF93
:1032E800EDC0DEFFEEC0DEFF20EE06F0D251D9269B
:1032F800D351DA22DE6ADE6ADE6ADD6A20EE16F073
:10330800D251D926D351DA22DE6ADE6ADE6ADD6A54
:10331800D2C0D9FFD3C0DAFFC2C1DEFFC3C1DDFF0F
:10332800D2C0D9FFD3C0DAFF10EE06F0DE50E12696
:10333800DD50E22220EE02F0D251D926D351DA2212
:10334800E6CFDEFFE5CFDDFF0101BF511200655179
:103358006411631103E1020E625D10E320EE12F0C6
:103368006051D9266151DA22DE50625DDE50635920
:10337800DE506459DE50655901E22FD2020E8C6F7F
:1033880041D262C08AF063C08BF0D8908B316B6FEA
:103398008A316A6F6A518A276B518B2360C039F072
:1033A80061C03AF020EE1EF06051D9266151DA2250
:1033B800DECF6AF0DECF6BF0DECF6CF0DECF6DF0E3
:1033C8008AC06EF08BC06FF0090E706FD8906F33A3
:1033D8006E33702FFBD76E516A253B6E6F516B2190
:1033E8003C6E000E6C213D6E000E6D213E6EF5ECBC
:1033F8004BF000018C6F8C5101E004D26A69010E18
:103408006B6F8AC06CF08BC06DF06A516C176B5192
:103418006D1760C06EF061C06FF06C516E276D5112
:103428006F232E0E6E258D6F000E6F218E6F8A4BC7
:103438008B2B62B104D066C086F0876B1AD06651B8
:103448006A6F6B6B6A3B6B3BF00E6B176A510F0B25
:103458006B13F00E6A178DC0D9FF8EC0DAFFDF50EC
:103468000F0B6C6F6D6B6A516C11866F6B516D1120
:10347800876F8DC0D9FF8EC0DAFF86C0DFFF20EED0
:1034880004F06051D9266151DA22010EDF6E60C066
:1034980039F061C03AF020EE1EF06051D926615132
:1034A800DA22DECF6AF0DECF6BF0DECF6CF0DECF53
:1034B8006DF08AC06EF08BC06FF0090E706FD890F7
:1034C8006F336E33702FFBD76E516A253B6E6F5189
:1034D8006B213C6E000E6C213D6E000E6D213E6E20
:1034E800F5EC4BF000018C6F8C5101E08BD16A69CF
:1034F800010E6B6F8AC06CF08BC06DF06A516C174F
:103508006B516D1760C06EF061C06FF06C516E2723
:103518006D516F232E0E6E258D6F000E6F218E6FED
:1035280062B10CD067C06AF00F0E6A178DC0D9FF60
:103538008EC0DAFFDF50F00B6A1112D066C06AF055
:1035480067C06BF068C06CF069C06DF0050E05D0FF
:10355800D8906D336C336B336A33E82EF9D76A51E0
:10356800886F896B8DC0D9FF8EC0DAFF88C0DFFFF6
:103578002BD160C039F061C03AF020EE1EF06051E6
:10358800D9266151DA22DECF6AF0DECF6BF0DECFCA
:103598006CF0DECF6DF063516E6F64516F6F6551E3
:1035A800706F716B6A516E253B6E6B516F213C6E6B
:1035B8006C5170213D6E6D5171213E6EF5EC4BF0F2
:1035C80000018C6F8C5101E01DD16A69010E6B6F8F
:1035D80062C06CF063C06DF0D8906C376D376A517B
:1035E8006C176B516D1760C06EF061C06FF06C5155
:1035F8006E276D516F232E0E6E258D6F000E6F2175
:103608008E6F8DC0D9FF8EC0DAFF66C0DFFF20EE57
:1036180001F08D51D9268E51DA2267C0DFFFD4D050
:1036280060C039F061C03AF020EE1EF06051D92632
:103638006151DA22DECF6AF0DECF6BF0DECF6CF0BC
:10364800DECF6DF062C06EF063C06FF064C070F0E2
:1036580065C071F0080E05D0D890713370336F33A0
:103668006E33E82EF9D76A516E253B6E6B516F2188
:103678003C6E6C5170213D6E6D5171213E6EF5ECC2
:103688004BF000018C6F8C5101E0BCD06A69010ECF
:103698006B6F62C06CF063C06DF0D8906C376D379B
:1036A800D8906C376D376A516C176B516D1760C0C5
:1036B8006EF061C06FF06C516E276D516F232E0E46
:1036C8006E258D6F000E6F218E6F20EE01F08D51EB
:1036D800D9268E51DA22DF506B6F6A6B20EE02F02A
:1036E8008D51D9268E51DA22DF506C6F6CC06DF087
:1036F8006E6B6F6B706B6EC070F06DC06FF06E6B41
:103708006D6B20EE03F08D51D9268E51DA22DF50F1
:10371800716F71C072F0736B746B756B72C075F0FA
:10372800746B736B726B6D517211766F6E5173118E
:10373800776F6F517411786F70517511796F6A5185
:1037480076117A6F6B5177117B6F000E78117C6F51
:10375800000E79117D6F8DC0D9FF8EC0DAFFDF5062
:103768007A117E6F7B517F6F7C51806F7D51816FA5
:10377800826B836B846BF00E8115856F82516613A3
:103788008351671384516813855169138DC0D9FF1C
:103798008EC0DAFF66C0DFFF20EE01F08D51D9261A
:1037A8008E51DA2267C0DFFF20EE02F08D51D92654
:1037B8008E51DA2268C0DFFF20EE03F08D51D92642
:1037C8008E51DA2269C0DFFF20EE04F06051D9265D
:1037D8006151DA22010EDF6E15D060C0D9FF61C0D9
:1037E800DAFFDF506A6F6B6B6B5101E0C7D56A5126
:1037F800010A01E1C6D5030A01E1BBD6010A01E1CC
:103808000FD7BCD58C51120049504810471003E11E
:10381800020E465C0FE320EE12F04450D9264550C4
:10382800DA22DE50465CDE504758DE504858DE50FB
:10383800495808E3010E00017C6F000E7D6B7E6B1A
:103848007F6BEFD100017C697D697E697F69D4D186
:1038580046C080F047C081F0D8908131616F8031D7
:10386800606F605180276151812344C039F045C0A1
:103878003AF020EE1EF04450D9264550DA22DECF29
:1038880060F0DECF61F0DECF62F0DECF63F080C0A3
:1038980064F081C065F0090E666FD89065336433B3
:1038A800662FFBD7645160253B6E655161213C6EE4
:1038B800000E62213D6E000E63213E6EF5EC4BF06A
:1038C800000901E0AED100016069010E616F80C09E
:1038D80062F081C063F0605162176151631744C0A0
:1038E80064F045C065F062516427635165232E0E6C
:1038F8006425D96E000E6521DA6EDF507A6F7B6B16
:10390800804B812B44C039F045C03AF020EE1EF0C0
:103918004450D9264550DA22DECF60F0DECF61F080
:10392800DECF62F0DECF63F080C064F081C065F066
:10393800090E666FD89065336433662FFBD76451E0
:1039480060253B6E655161213C6E000E62213D6E23
:10395800000E63213E6EF5EC4BF0000901E061D1E9
:1039680000016069010E616F80C062F081C063F080
:10397800605162176151631744C064F045C065F037
:1039880062516427635165232E0E6425D96E000E9B
:103998006521DA6EDF50676F666B66517A1367517F
:1039A8007B1346B006D07A51786F0F0E7B15796F6E
:1039B8000FD07AC060F07BC061F0040E626FD890BF
:1039C80061336033622FFBD760C078F061C079F053
:1039D80078C07CF079C07DF05BD044C039F045C038
:1039E8003AF020EE1EF04450D9264550DA22DECFB8
:1039F80060F0DECF61F0DECF62F0DECF63F04750DB
:103A0800646F4850656F4950666F676B60516425F5
:103A18003B6E615165213C6E625166213D6E63517A
:103A280067213E6EF5EC4BF0000901E0FAD0000189
:103A38006069010E616F46C062F047C063F0D890BC
:103A480062376337605162176151631744C064F08D
:103A580045C065F062516427635165232E0E6425C5
:103A6800826F000E6521836F20EE01F08251D92606
:103A78008351DA22DF50616F606B82C0D9FF83C047
:103A8800DAFFDF506013000E60C07CF061C07DF08B
:103A98007E6B7F6BC6D044C039F045C03AF020EE4B
:103AA8001EF04450D9264550DA22DECF60F0DECF32
:103AB80061F0DECF62F0DECF63F046C064F047C04D
:103AC80065F048C066F049C067F0080E05D0D89088
:103AD8006733663365336433E82EF9D7605164255C
:103AE8003B6E615165213C6E625166213D6E6351AA
:103AF80067213E6EF5EC4BF0000901E092D0000121
:103B08006069010E616F46C062F047C063F0D890EB
:103B180062376337D89062376337605162176151F3
:103B2800631744C064F045C065F06251642763516F
:103B380065232E0E6425826F000E6521836F20EEAB
:103B480001F08251D9268351DA22DF50616F606B10
:103B580020EE02F08251D9268351DA22DF50626FBB
:103B680062C063F0646B656B666B64C066F063C0CB
:103B780065F0646B636B20EE03F08251D9268351A4
:103B8800DA22DF50676F67C068F0696B6A6B6B6B2E
:103B980068C06BF06A6B696B686B635168116C6F16
:103BA800645169116D6F65516A116E6F66516B11C1
:103BB8006F6F60516C11706F61516D11716F000EF4
:103BC8006E11726F000E6F11736F82C0D9FF83C0C0
:103BD800DAFFDF507011746F7151756F7251766F23
:103BE8007351776F74517C6F75517D6F76517E6F0D
:103BF8000F0E77157F6F15D044C0D9FF45C0DAFF87
:103C0800DF50606F616B615101E014D66051010AA9
:103C180001E11ED6030A01E1E0D6010A01E13BD722
:103C280009D67CC044F07DC045F07EC046F07FC018
:103C380047F012002A6E1BC041F01CC042F02A5007
:103C480001E0040C010E3F6E54B0030CE9D1B2EC54
:103C580056F0000901E1FDD13F6AFBD1146A156AEB
:103C6800166A176A090EC2EC54F0000901E0F1D196
:103C78002B0E0B6E0C6A0E6A100E0D6E3AEC51F09C
:103C8800000901E1E6D12B44E846030BE8064DE1C3
:103C980032C01DF03F0E1D161DC01EF01F6A206A9F
:103CA800216A1FC021F01EC020F01F6A1E6A33500F
:103CB800236E226A3450246E256A2250242623500B
:103CC800252224501E24266E25501F20276E000E04
:103CD8002020286E000E2120296E26283B6E000E1B
:103CE80027203C6E000E28203D6E000E29203E6ED7
:103CF8003BC01DF03CC01EF03DC01FF03EC020F090
:103D08000A0ED8901D361E361F362036E82EF9D7F3
:103D18001BC0D9FF1CC0DAFF1DC0DEFF1EC0DEFFBE
:103D28001FC0DEFF20C0DEFF97D71D6A35AE01D069
:103D38001D2A010E1D1630C01EF00F0E1E1634501F
:103D4800030B020DF3501E241D24020F406E315048
:103D5800030B1D6E1E6A0A0ED8901D361E36E82EFD
:103D6800FBD732501F6E206AD8901F362036D89065
:103D78001F3620363344E846030B216E226A1F5053
:103D88002126205022221D5021261E502222212A7F
:103D9800000E222221C03BF022C03CF03D6A3E6A60
:103DA80040C01DF0F70E1D263BC01EF03CC01FF0A2
:103DB8003DC020F03EC021F01D2A05D0D8901E3607
:103DC8001F36203621361D2EF9D734D051A43FD0C6
:103DD800146A156A166A176A8D0EC2EC54F0000947
:103DE80001E037D104EC57F02B0E0B6E0C6A0E6A0B
:103DF800100E0D6E3AEC51F0000901E12AD1300E97
:103E0800406E03D004EC57F040064050FBE135C04B
:103E18001DF01D3A0F0E1D16100E1E6E1F6A206A29
:103E2800216A1D2A05D0D8901E361F362036213625
:103E38001D2EF9D71BC0D9FF1CC0DAFF1EC0DEFF3C
:103E48001FC0DEFF20C0DEFF21C0DEFF05D7146AD9
:103E5800156A166A176A090EC2EC54F0000901E0E7
:103E6800F8D02B0E0B6E0C6A0E6A100E0D6E3AEC23
:103E780051F0000901E1EDD051A232D038C01DF057
:103E8800060E1E6ED8901D321E2EFCD7FF0E1D2664
:103E980035503F0B1F6E206AD8901F3620363644A7
:103EA800010B1F26000E20221F2A20221D2A03D0C4
:103EB800D8901F3620361D2EFBD71F50216E20505C
:103EC800226E236A246A1BC0D9FF1CC0DAFF21C0F6
:103ED800DEFF22C0DEFF23C0DEFF24C0DEFFBCD62B
:103EE8003650030B1D6E1E6AD8901D361E36D890AC
:103EF8001D361E36D8901D361E363638E842070B5A
:103F08001D26000E1E221D2A1E223540E8423F0BA8
:103F18001F0B1F6E206A1F2A000E20221D501F0231
:103F2800F3CF21F0F4CF22F02002F35022261E50C6
:103F38001F02F35022262150236E2250246E256A38
:103F4800266A1BC0D9FF1CC0DAFF23C0DEFF24C0CD
:103F5800DEFF25C0DEFF26C0DEFF7ED641C0D9FFCA
:103F680042C0DAFF51C0DFFF77D6146A156A166AB5
:103F7800176A090EC2EC54F000096BE141C00BF05E
:103F880042C00CF00E6A100E0D6E3AEC51F00009AA
:103F980001E062D65ED0146A156A166A176A0A0EBC
:103FA800C2EC54F0000955E141C00BF042C00CF0DE
:103FB8000E6A100E0D6E3AEC51F0E9D7146A156AC4
:103FC800166A176A3A0EC2EC54F0000942E1040E70
:103FD800406E0AD004EC57F041C0D9FF42C0DAFF66
:103FE800DF6E414A422A4006405001E135D6F2D7F9
:103FF800146A156A166A176A8D0EC2EC54F0000925
:1040080028E104EC57F041C00BF042C00CF00E6AF6
:10401800400E0D6E3AEC51F0BAD7040E3F6E19D02F
:104028001A501D6E1E6A1E50F8E11D5001E10FD690
:10403800010A01E113D6020A01E1C8D6090A8EE095
:10404800010A93E0070AA7E0010AB8E0030AD0E0F2
:10405800E4D71BEC57F03F5012006AC06DF06BC0FC
:104068006EF001017E6B7F6BF8D169C046F06D0E72
:10407800476E6CC048F04750D96EDA6ADECFF6FF5B
:10408800DDCFF7FFF86A000EF86E0800F550250A34
:10409800D8A4C5D14750D96EDA6ADE2A000EDD22CF
:1040A8000101806B816B846B856B826983694750E2
:1040B800D96EDA6ADECFF6FFDDCFF7FFF86A000EB9
:1040C800F86E0800F550780AD8B40FD04750D96E6A
:1040D800DA6ADECFF6FFDDCFF7FFF86A000EF86E7A
:1040E8000800F550580AD8A470D14750D96EDA6A3A
:1040F800DECFF6FFDDCFF7FFF86A000EF86E080096
:10410800F5CF68F04750D96EDA6ADE2A000EDD2254
:104118004850D96EDA6ADF50DF2ADF2AD96EDA6AA8
:10412800DECF49F0DDCF4AF049C060F04AC061F007
:104138000001626B636B646B656B666B676B46C093
:1041480024F060C025F061C026F062C027F063C08B
:1041580028F064C029F065C02AF066C02BF067C05B
:104168002CF068C02DF0010183BF01D0849383BF78
:1041780005D0835107E18205D8B004D0376A010E13
:10418800366E04D082C136F083C137F080C140F06A
:1041980081C141F084A904D0FE0E4026FF0E4122C1
:1041A80025C038F026C039F027C03AF028C03BF0C7
:1041B80029C03CF02AC03DF02BC03EF02CC03FF097
:1041C800436A1F0E426E02019F6B6DD04206D8A053
:1041D80043060F0E3814446E456A45BE08D0455054
:1041E80004E10A0E445CD8A002D0570E01D0300E6C
:1041F8004426000E4522BF0E2E6E2F682D50306EBD
:10420800316A2E5030262F503122315005E11A0ED6
:10421800305C02E2010E01D0000E326E336A325079
:104228003310D8B425D09F0E2E6E2F68200E441060
:10423800306E000E4510316E2E5030262F50312230
:10424800315005E11A0E305C02E2010E01D0000E79
:10425800346E356A34503510D8B40AD044C011F0E1
:1042680045C012F06CEC53F011C044F012C045F098
:10427800800E4224D96E020E4320DA6E44C0DFFF5E
:104288003606D8A037064006D8A04106040E2E6E82
:10429800D8903F323E323D323C323B323A323932AC
:1042A80038322E2EF5D743BE21D0435004E1020EFA
:1042B800425CD8A01BD0385039103A103B103C1043
:1042C8003D103E103F10D8A481D737BE05D03750D7
:1042D80002E13604D8B07AD741BE08D0415003E194
:1042E8004004D8A003D0010184B370D7010184A988
:1042F80016D04206D8A04306800E4224D96E020E7C
:104308004320DA6E2DC0DFFF4206D8A04306800E98
:104318004224D96E020E4320DA6E300EDF6E24C0BE
:104328001AF0800E42241B6E020E43201C6E40C001
:104338001DF041C01EF084A108D01BC014F01CC0A1
:1043480015F01AC016F0BDEC55F01EBE05D01DC004
:1043580022F01EC023F002D0226A236A206A216A52
:104368000AD0000E0D6E200E0C6E1AC00EF0F3EC83
:104378004DF0204A212A2250205C2150800A1F6ECD
:104388002350800A1F58D8A0ECD7010184B108D067
:104398001BC014F01CC015F01AC016F0BDEC55F087
:1043A8001BC00BF01CC00CF0D0EC53F022500B24B7
:1043B8001A6E23500C201B6E1AC024F01BC025F067
:1043C80024C046F025C047F043D04750D96EDA6A7A
:1043D800DECFF6FFDDCFF7FFF86A000EF86E0800B3
:1043E800F550250AD8A412D04750D96EDA6ADE2AC9
:1043F800000EDD22000E0D6E250E0C6E46C00EF06E
:10440800F3EC4DF0476A010E466E22D04750D96E44
:10441800DA6ADE2A000EDD22466A476A19D047505A
:10442800D96EDA6ADECFF6FFDDCFF7FFF86A000E45
:10443800F86E0800F5500C6E0D6A46C00EF0F3ECED
:104448004DF04750D96EDA6ADE2A000EDD22DAD73F
:10445800465001017E2747507F236DC0F6FF6EC08E
:10446800F7FF0800F55001E000D67EC169F07FC172
:104478006AF012000001896F495002E034EC4FF0F5
:104488000001886B485001E195D1899F040E891974
:1044980003E0140E891907E10101866B876B496AED
:1044A800070E486E070C3F0E891907E14D6A010196
:1044B800866B876B486A496A12005F0E891907E1A3
:1044C8000101956B866B876B486A496A12003F0E3B
:1044D800896506D05F0E896103D0400E8919F0E125
:1044E800400E89190AE1010E0101956F4D6A01011B
:1044F800866B876B486A496A1200200E891901E0A9
:1045080059D1010E4D6EF3D7600E89190AE10101E8
:10451800955107E09351080ED8B4030E0001886F37
:104528007ED0600E0001891909E14D5007E00101B4
:10453800935102E0090E15D0050E13D0680E8919A3
:1045480009E14D5007E01A0E0101876F900E24D142
:1045580083808AD1680E891907E10101955104E029
:10456800020E0001886F5BD06A0E0001891907E10D
:104578004D5005E01A0E0101876FF40E0DD16C0E37
:10458800891907E14D5005E01A0E0101876F2C0EBD
:1045980003D1700E89190AE10101955107E0040E53
:1045A8000001886F0101866B876BD2D7700E0001FE
:1045B800891901E059D14D5001E156D11B0E010175
:1045C800876F620EE9D08380020E891905E11A0E01
:1045D8000101876F920E866F050E0001891905E1AA
:1045E8001A0E0101876FAE0E866F070E000189193A
:1045F80005E11A0E0101876FB80E866F080E0001DB
:10460800891905E11A0E0101876FCC0E866F030E1A
:104618000001891902E0892906E1886B839001016C
:10462800866B876B21D1160E891901E01DD11A0EF0
:104638000101876FA40EA0D0050E891901E014D1DD
:104648001A0E0101876FF50E97D089C050F01A0E27
:104658000101876F9B0E90D01A0E0101876F9C0E87
:104668008BD05050070D500EF324D96E010EF42054
:10467800DA6E89C0DFFF1A0E0101876F9D0E7CD0AC
:104688005050070D510EF324D96E010EF420DA6E46
:1046980089C0DFFF1A0E0101876F9E0E6DD0505042
:1046A800070D520EF324D96E010EF420DA6E89C07C
:1046B800DFFF0101866B876B010E2AD01A0E0101FC
:1046C800876FB90E69D01A0E0101876FBA0E54D0E0
:1046D8001A0E0101876FBB0E866FA10E0001606F75
:1046E800FE0E616FE0EC56F00101946B866B876BF0
:1046F8004BD00101866B876BA10E0001606FFE0E27
:10470800616FE0EC56F040D00101866B876B060EB6
:104718000001886FA9D089C050F00101866B876BB2
:104728000001886B31D00101936B1A0E876FF70E69
:10473800866F2AD01A0E0101876FF70E1DD083905D
:10474800270E0101876F0F0E17D0180E891901E087
:104758008BD01A0E0101876F2D0E0ED01A0E010193
:10476800876F2E0E09D01A0E0101876F2F0E04D005
:104778001A0E0101876F300E866F76D00101866BA5
:10478800876B0A0E0001886F83906ED0040E886FC5
:10479800270E0101876F0F0E866FDAD6838001011D
:1047A80004D08390010E0101936F866B876B000123
:1047B800886B5AD086C186F087C187F0875107E099
:1047C8001A0A09E0010A48E03C0A4CE04DD086513B
:1047D80001E19AD649D086512C0AB7E0010ABEE019
:1047E800030AC1E0010AC4E01F0AC8E0A00A01E107
:1047F800EAD6020A01E129D7090A01E12DD7070AF9
:1048080001E12FD7010A01E13BD7030A01E147D7AC
:104818003A0A01E179D70A0AC4E0160A01E14ED73B
:10482800010A01E150D7030A01E152D7010A01E167
:1048380060D7790A01E194D60E0A01E16CD7380AEB
:1048480001E1FAD6010A01E16ED7030A01E172D744
:10485800010A01E174D708D08651580A97E03A0A4C
:104868009DE002D086510F0A88C048F0496A1200BC
:1048780020EE04F0A651D926A751DA22DECFAAF0FD
:10488800DDCFABF0AA29B36F000EAB21B46FB31123
:10489800D8B4040C20EE0EF0A651D926A751DA227E
:1048A800DE50DE10DE10DE1001E1040CB3C0AAF009
:1048B8000F0EAA1701E094D120EE0EF0A651D926CA
:1048C800A751DA22DE2A000EDE22DE22DE2220EEC8
:1048D8000AF0A651D926A751DA22DE50DE10DE10E2
:1048E800DE1011E1A6C0D9FFA7C0DAFF10EE08F06C
:1048F800DE50E126DD50E222E650B35DE650B459C1
:1049080001E26ED1040CB3C0AAF0B4C0ABF0040E3F
:10491800AC6FD890AB33AA33AC2FFBD7AD69AE6977
:10492800A6C0D9FFA7C0DAFF10EE02F0DE50E126DC
:10493800DD50E222E750AF6FB06BAD51AF27AE51FB
:10494800B023AA51AF17AB51B017AF51B01101E066
:1049580047D1A6C0D9FFA7C0DAFFDECF44F0DDCF2C
:1049680045F020EE0AF0A651D926A751DA22DECF6B
:1049780046F0DECF47F0DECF48F0DECF49F008EC56
:104988001CF044C0B5F045C0B6F046C0B7F047C00B
:10499800B8F00001B851B711B61104E1020EB55DC7
:1049A80001E2020CB52907E1B62905E1B72903E1BF
:1049B800B82901E1010CA6C0D9FFA7C0DAFF10EEA3
:1049C80012F0DE50E126DD50E222E650B55DE650F9
:1049D800B659E650B759E650B85901E2D2D0A851B5
:1049E800A91101E1040CA6C0D9FFA7C0DAFFDECFE8
:1049F8008FF0DDCF90F020EE0AF0A651D926A7510E
:104A0800DA22DECF91F0DECF92F0DECF93F0DECF68
:104A180094F0E9EC2FF08FC0B5F090C0B6F091C0DB
:104A2800B7F092C0B8F0B551B611B711B81101E19D
:104A3800070CB505B611B711B81101E1020CB5297B
:104A480007E1B62905E1B72903E1B82901E1010C1D
:104A5800A6C0D9FFA7C0DAFFDECF24F0DDCF25F04E
:104A6800C2EC40F0000901E0010CA6C0D9FFA7C0C4
:104A7800DAFFDECFAAF0DDCFABF02E0E0001AA25BB
:104A88000B6E000EAB210C6E0E6A0D6A020E106ED4
:104A98000F6A16EC56F0A6C0D9FFA7C0DAFFDECF22
:104AA8000BF0DDCF0CF0B5C00DF0B6C00EF0B7C0FE
:104AB8000FF0B8C010F0F0EC45F0A6C0D9FFA7C0C1
:104AC800DAFF10EE2AF0DE50E126DD50E2220BC0BC
:104AD800E6FF0CC0E6FF0DC0E6FF0EC0E6FF0001D2
:104AE800B16BB26B2BD0A6C0D9FFA7C0DAFF10EE0E
:104AF80004F0DE50E126DD50E222010EE76EA6C08A
:104B0800D9FFA7C0DAFFDECF24F0DDCF25F0C2EC55
:104B180040F0000901E0010CA6C0D9FFA7C0DAFFE8
:104B280010EE2AF0DE50E126DD50E222E62A000EE1
:104B3800E622E622E6220001B14BB22BA6C0D9FF3D
:104B4800A7C0DAFF10EE02F0DE50E126DD50E222C7
:104B5800E750AA6FAB6BAA51B15DAB51B259C3E331
:104B6800A6C0D9FFA7C0DAFF10EE2AF0DE50E12672
:104B7800DD50E222B151E65EB251E65A000EE65A25
:104B8800E65A20EE0AF0A651D926A751DA22B5C076
:104B9800DEFFB6C0DEFFB7C0DEFFB8C0DEFFA6C0CE
:104BA800D9FFA7C0DAFFDECF0BF0DDCF0CF0B5C020
:104BB8000DF0B6C00EF0B7C00FF0B8C010F0F0ECB2
:104BC80045F0000120EE0EF0A651D926A751DA22B1
:104BD8000BC0DEFF0CC0DEFF0DC0DEFF0EC0DEFF27
:104BE80020EE04F0A651D926A751DA22B3C0DEFF81
:104BF800B4C0DDFF0F0EB315AA6FAB6B050ED890CE
:104C0800AA37AB37E82EFBD7A6C0D9FFA7C0DAFF73
:104C1800DECFACF0DDCFADF0AA51AC27AB51AD2360
:104C28002E0EAC27000EAD2320EE12F0A651D92689
:104C3800A751DA22ACC0DEFFADC0DDFF000C000ECC
:104C4800846F020E856F340E866F0A0E876F020E10
:104C5800896F886BDD0E8A6F8B6BFEEC11F0FF6F2E
:104C6800EE0E606FFD0E616FDDC062F0DEC063F0B6
:104C7800E0EC56F00001DF6BE06BDB6BDC6BE16BAB
:104C8800E26BE151BD0FD96EDA6ADF6AE151CC0FF0
:104C9800D96EDA6A000EDF6EE14BE22BE2BFF1D784
:104CA800E25103E10F0EE15DECE3E36BE46B30D11D
:104CB800340EE325D96E0A0EE421DA6E0D0EDE18E5
:104CC80001E0EBD08B0E0B6EFF0E0C6EBD0E0D6E61
:104CD8008EEC4CF00B500C1007E1CC0E126E77ECFA
:104CE80046F012500101FB6F850E0B6EFF0E0C6E25
:104CF800BD0E0D6E8EEC4CF00B500C1007E1CC0E77
:104D0800126E77EC46F0125001019F6F6A0E0B6E1F
:104D1800FF0E0C6EBD0E0D6E8EEC4CF00B500C1091
:104D280007E1CC0E126E77EC46F0125001019B6F32
:104D3800D00E0B6EFF0E0C6EBD0E0D6E8EEC4CF091
:104D48000B500C1007E1CC0E126E77EC46F01250A7
:104D58000101996FD40E0B6EFF0E0C6EBD0E0D6E19
:104D68008EEC4CF00B500C1007E1CC0E126E77EC69
:104D780046F012500101ED6F0001E56BE66BAE0ED7
:104D88006F6F706B710E716FFF0E726FE5C073F00D
:104D9800E6C074F06CEC54F0AE0E0B6E0C6ABD0EEF
:104DA8000D6E8EEC4CF00B500C1018E10F0E00013C
:104DB800E503F3CFACF0F4CFADF0E603F350AD2745
:104DC800340EAC250B6E0C0EAD210C6ECC0E0D6E98
:104DD8000E6A106A0F0E0F6E96EC51F00001E54B4B
:104DE800E62BE6BFCCD7E65103E1100EE55DC7E33D
:104DF800E66B010EE56FAE0E6F6F706B780E716F1C
:104E0800FF0E726FE5C073F0E6C074F06CEC54F0FE
:104E1800AE0E0B6E0C6ABD0E0D6E8EEC4CF00B5088
:104E28000C1018E10F0E0001E503F3CFACF0F4CF3E
:104E3800ADF0E603F350AD27240EAC250B6E0D0E36
:104E4800AD210C6ECC0E0D6E0E6A106A0F0E0F6E31
:104E580096EC51F00001E54BE62BE6BFCCD7E651C6
:104E680003E1040EE55DC7E3E16BE26BE151BD0FC1
:104E7800D96EDA6ADF6AE151CC0FD96EDA6A000EB0
:104E8800DF6EE14BE22BE2BFF1D7E25103E10F0EF7
:104E9800E15DECE3DB6BDC6B15D0340EE325D96EFA
:104EA8000A0EE421DA6E0A0EDE1830E0340EE3252D
:104EB800D96E0A0EE421DA6E200EDE1806E1DC6BEC
:104EC800010EDB6FDF6BE06B21D0DB51DC1109E0F9
:104ED800340EE325D96E0A0EE421DA6EDF51CC0FC9
:104EE80008D0340EE325D96E0A0EE421DA6EDF51BC
:104EF800BD0FE16EE26ADFCFE7FFE0BF05D0E0510A
:104F080005E10F0EDF5D02E2DF4BE02BE34BE42B04
:104F1800DD51E35DDE51E45901E2CAD6DE0E606F71
:104F2800FD0E616F9BC162F0636BE0EC56F0490EB9
:104F38000001606FFE0E616FFBC162F0636BE0EC15
:104F480056F03A0E0001606FFE0E616F9FC162F06D
:104F5800636BE0EC56F00001E56BE66B7C0E606F6E
:104F6800FD0E616FE5C062F0E6C063F00F0EE50369
:104F7800F3CFACF0F4CFADF0E603F350AD27340E29
:104F8800AC25646F0C0EAD21656FE0EC56F00001A6
:104F9800E54BE62BE6BFE2D7E65103E1100EE55DEF
:104FA800DDE3E46B010EE36F8D0E606FFD0E616F44
:104FB800E3C062F0E4C063F00F0EE303F3CFACF09C
:104FC800F4CFADF0E403F350AD27240EAC25646FA5
:104FD8000D0EAD21656FE0EC56F00001E34BE42BBC
:104FE800E4BFE2D7E45103E1040EE35DDDE39E0E86
:104FF800606FFB0E616FE0EF56F018C0F6FF19C046
:10500800F7FF0800F5CF46F0184A192A465001E183
:105018001200250E461804E04650D5EC56F0EDD7A0
:10502800416A426A18C0F6FF19C0F7FF0800F5CFB9
:1050380046F0184A192A300E46180DE1426A010E48
:10504800416E18C0F6FF19C0F7FF0800F5CF46F00B
:10505800184A192A06D02D0E461803E1426A020E94
:10506800EFD7396A3A6A1CD00A0E3902F3CF1BF01F
:10507800F4CF1CF03A02F3501C2646501B26000EB3
:105088001C22D00E1B24396EFF0E1C203A6E18C04D
:10509800F6FF19C0F7FF0800F5CF46F0184A192A9D
:1050A8002F0E466403D0390E4664DED76C0E4618C0
:1050B80003E04C0E46180AE1418418C0F6FF19C0F7
:1050C800F7FF0800F5CF46F0184A192A465001E1C3
:1050D800120046C045F0600E456472D0200E455E51
:1050E8006FD01A50D96EDA6A020EDF26DF5CD96EED
:1050F800DA6ADECF35F0DECF36F03B6A3C6A02D0A2
:105108003B4A3C2A3B5035241B6E3C5036201C6ED3
:105118001BC0F6FF1CC0F7FF000EF86E0E0EF764FA
:1051280003D00800F55005D0F6CFE9FFF7CFEAFF26
:10513800EF50000904E0E4D7200ED5EC56F041B258
:105148000BD03B501B6E3C501C6E3B4A3C2A3950DE
:105158001B5C3A501C58F0E335C00CF036C00DF01B
:10516800EBEC51F003D0200ED5EC56F03B501B6E03
:105178003C501C6E3B4A3C2A39501B5C3A501C5828
:1051880001E33BD7F0D71A50D96EDA6ADF50DF2A2D
:10519800DF2AD96EDA6ADF50D5EC56F02ED7386A96
:1051A800020E08D0386A080E05D0386A0A0E02D0F6
:1051B800386A100E376E19D04650D5EC56F01DD708
:1051C80045501B6E1C6A1C50F7E11B50420AE7E071
:1051D800010AD9E0070AE9E00B0AE4E01C0A81E0C9
:1051E800060AE3E00D0AE4E0E7D741B430D0440E04
:1051F800451813E01A50D96EDA6ADF50DF2ADF2A21
:10520800D96EDA6ADECF1BF0DDCF1CF01BC02DF0A3
:105218001CC02EF02F6A306A11D01A50D96EDA6A83
:10522800DF50DF2ADF2AD96EDA6ADECF2DF0DDCF34
:105238002EF0000E2EBEFF0E2F6E306E2DC03DF0EC
:105248002EC03EF02FC03FF030C040F010D01A50B2
:10525800D96EDA6A040EDF26DF5CD96EDA6ADECF31
:105268003DF0DECF3EF0DECF3FF0DECF40F0440E23
:1052780045180CE140AE0AD03D6C3E1ED8B03E2A1F
:105288003F1ED8B03F2A000E40564186436A446A02
:105298003DC00BF03EC00CF03FC00DF040C00EF01A
:1052A80037C00FF038C010F0116A126A7CEC50F069
:1052B8000B50456E3DC00BF03EC00CF03FC00DF0EA
:1052C80040C00EF037C00FF038C010F0116A126AF3
:1052D800F9EC4EF00BC03DF00CC03EF00DC03FF0B5
:1052E8000EC040F0090E45640BD0780E461803E056
:1052F800326A070E02D0326A270E316E31504526C7
:1053080043501D0FD96EDA6A4550300FDF6E434A9D
:10531800442A3D503E103F10401005E0445003E140
:10532800100E435CB5E341A608D043501D0FD96E5B
:10533800DA6A2D0EDF6E434A442A43C03BF044C06C
:105348003CF041B003D0346A200E02D0346A300EEB
:10535800336E33C045F003D04550D5EC56F041B21A
:105368000BD03B501B6E3C501C6E3B4A3C2A3950BC
:105378001B5C3A501C58F0E34306D8A0440643503F
:105388001D0FD96EDA6ADF50D5EC56F04350441041
:1053980004E0F2D7200ED5EC56F03B501B6E3C5083
:1053A8001C6E3B4A3C2A39501B5C3A501C5801E39E
:1053B80024D6F0D7000E0001F66F0A0EF56F000E26
:1053C800F46F050EF36F8ED1F66B140EF56F82D164
:1053D800FD0E0C6EFC0E0D6EEBEC51F08FB204D08E
:1053E8000001F66B1E0EF56F090E0001F26F1E0E1E
:1053F800F16FE40EE82EFED7F12FFCD7F22FFAD783
:1054080000F068D1EF0E0C6EFE0E0D6EEBEC51F055
:10541800060E0001D26F080ED36FA00ED46FFB0EDC
:10542800D56FD66B43EC4CF0FF6FFF513EEC52F05A
:105438000001FF51D9E1F66B230ED5D7580E0C6E3B
:10544800FE0E0D6EEBEC51F0000E0001D26F020E55
:10545800D36F120ED46FFF0ED56F010ED66F48ECC6
:1054680017F00001FF6FFF513EEC52F00001FF51B1
:105478000AE123EC26F0000E486E020E496E14EC89
:1054880055F00001FF6FFF513EEC52F0000E000195
:10549800F66F250EF56F01019B510DE1F96B340E86
:1054A80000016F6F0C0E706FD50E716FFE0E726F6C
:1054B8006CEC54F00DD0060E0001606FFC0E616FAD
:1054C8009BC162F0636BF9C164F0656BE0EC56F068
:1054D800670E0001606FFE0E616F0101F9510F0D3B
:1054E800340EF3240001626F0C0EF420636FE0ECBD
:1054F80056F07AD76B0E0C6EFD0E0D6EEBEC51F07C
:10550800000E0001D26F020ED36FC80ED46FFE0ECC
:10551800D56F010ED66F48EC17F00001FF6FFF51F1
:105528003EEC52F00001FF510AE118EC37F0000E92
:10553800486E020E496E14EC55F00001FF6FFF51E2
:105548003EEC52F0000E0001F66F280EF56F0101D7
:105558009B510DE1F96B340E00016F6F0C0E706FEB
:10556800D50E716FFE0E726F6CEC54F00DD0060EF6
:105578000001606FFC0E616F9BC162F0636BF9C143
:1055880064F0656BE0EC56F0670E0001606FFE0E8C
:10559800616F0101F9510F0D340EF3240001626FA0
:1055A8000C0EF420636FE0EC56F01ED7CF0E606F40
:1055B800FC0E616F0101F9510F0D340EF324000147
:1055C800626F0C0EF420636FE0EC56F0000E0001E1
:1055D800D26F020ED36F0101F9510F0D340EF3246F
:1055E8000001D46F0C0EF420D56F030ED66F48EC73
:1055F80017F00001FF6FFF513EEC52F00001FF5120
:1056080003E1F66B3C0EF56F040EFF1901E0ECD6D2
:10561800F66B320EE8D6370E606FFD0E616F010132
:10562800F9510F0D340EF3240001626F0C0EF420B3
:10563800636FE0EC56F0000E0001D26F020ED36FDC
:105648000101F9510F0D340EF3240001D46F0C0E33
:10565800F420D56F070ED66F48EC17F00001FF6FE6
:10566800FF5101E0C1D6F66B3C0EBDD6110E606F3E
:10567800FD0E616F0101F9510F0D340EF324000185
:10568800626F0C0EF420636FE0EC56F00001F06BD3
:10569800010EEF6F010CF5C0F1F0F6C0F2F0F25117
:1056A80019E1F1510A0A01E18FD61E0A01E190D6EB
:1056B8000A0A01E1A7D63D0A01E1C0D6060A01E1BE
:1056C80019D70D0A01E172D7050A04E01F0AA3E001
:1056D8000E0ACCE0140E0001F519F61103E0F307E9
:1056E800D8A0F407F4BF04D0F451D5E1F305D3E210
:1056F800EF6BF06B120043C024F044C025F0C2ECFD
:1057080040F0456E455001E08FD143C0D9FF44C0F9
:10571800DAFF030EDE1801E077D120EE05F04350E2
:10572800D9264450DA22DE0401E06ED12E0E43243D
:105738000B6E000E44200C6E0E6A0D6A020E106E7F
:105748000F6A16EC56F022EE2CF04350D92644503E
:10575800DA22550EDF6E22EE2DF04350D926445042
:10576800DA22AA0EDF6E20EE2EF04350D9264450DE
:10577800DA22520EDF6E20EE2FF04350D926445025
:10578800DA22520EDF6E20EE30F04350D926445014
:10579800DA22610EDF6E20EE31F04350D9264450F4
:1057A800DA22410EDF6E22EE12F04350D926445021
:1057B800DA22720EDF6E22EE13F04350D9264450DF
:1057C800DA22720EDF6E22EE14F04350D9264450CE
:1057D800DA22410EDF6E22EE15F04350D9264450EE
:1057E800DA22610EDF6E20EE0EF04350D9264450C7
:1057F800DA2212EE16F04350E1264450E222DFCFBF
:10580800E7FF22EE17F04350D9264450DA2210EE73
:105818000EF04350E1264450E222E6CF60F0E5CF97
:1058280061F061C060F00001616B6051DF6E22EED3
:1058380018F04350D9264450DA2210EE0EF04350A7
:10584800E1264450E222E6CF60F0E6CF61F0E6CFF1
:1058580062F0E6CF63F0110E05D0D890633362335F
:1058680061336033E82EF9D76051DF6E22EE19F00C
:105878004350D9264450DA2210EE0EF04350E12668
:105888004450E222E6CF60F0E6CF61F0E6CF62F066
:10589800E6CF63F0190E05D0D890633362336133D5
:1058A8006033E82EF9D76051DF6E20EE0AF04350DE
:1058B800D9264450DA2212EE1AF04350E126445019
:1058C800E222DFCFE7FF22EE1BF04350D9264450F7
:1058D800DA2210EE0AF04350E1264450E222E6CFE5
:1058E80060F0E5CF61F061C060F0616B6051DF6E20
:1058F80022EE1CF04350D9264450DA2210EE0AF06A
:105908004350E1264450E222E6CF60F0E6CF61F052
:10591800E6CF62F0E6CF63F0110E05D0D89063337E
:10592800623361336033E82EF9D76051DF6E22EEBF
:105938001DF04350D9264450DA2210EE0AF04350A5
:10594800E1264450E222E6CF60F0E6CF61F0E6CFF0
:1059580062F0E6CF63F0190E05D0D8906333623356
:1059680061336033E82EF9D76051DF6E20EE1AF00C
:105978004350D9264450DA22DECF60F0DECF61F002
:10598800DECF62F0DECF63F06029646F000E612124
:10599800656F000E6221666F000E6321676F20EE4F
:1059A8002AF04350D9264450DA2264C0DEFF65C08D
:1059B800DEFF66C0DEFF67C0DEFF2E0E43241A6ED0
:1059C800000E44201B6E20EE2AF04350D926445086
:1059D800DA22DECF1CF0DECF1DF0DECF1EF0DECFE8
:1059E8001FF0216A010E206E20EE01F04350D926E7
:1059F8004450DA22DF50E9EC47F020EE05F043503E
:105A0800D9264450DA22DF6A1A6A1B6A1C6A20EE19
:105A180001F04350D9264450DA22DF501EEC1EF024
:105A2800000902E0010E456E45501200838E838006
:105A380089EC3EF0CDC0B0F1CEC0B1F10101B0515A
:105A4800B1111AE05050140D130EF324D96E010E43
:105A5800F420DA6E5050140D130EF324E16E010E8B
:105A6800F420E26EE7500409DF6EA6EC55F0B0C1F1
:105A7800E4F0B1C1E5F0120099515BE05050140D0B
:105A8800070EF324D96E010EF420DA6E74C1EBF020
:105A980075C1ECF076C1EDF00001EA6B000EEA2565
:105AA800EE6F010EEB21EF6F000EEC21F06F000E90
:105AB800ED21F16FDE50EE193CE1DE50EF1939E1CE
:105AC800DE50F01936E1DE50F11933E116EC50F0F2
:105AD8000FC0B6F110C0B7F111C0B8F112C0B9F1DA
:105AE800000EE8CF34FA2AEE35F0B9C1DFFFE8CF6F
:105AF80036FA2AEE37F0B8C1DFFFE8CF38FA2AEED7
:105B080039F0B7C1DFFFE8CF3AFA2AEE3BF0B6C169
:105B1800DFFF0101FA93010E496E486A92EC32F0F8
:105B28000101FA934E6A83904EC0E4F00001E56BE0
:105B380012005050140D0F0EF324D96E010EF420EC
:105B4800DA6EDECFE6F0DECFE7F0DECFE8F0DECFCC
:105B5800E9F0E7C0E6F0E8C0E7F0E9C0E8F00001E6
:105B6800E96BE6C0ABF1E7C0ACF15050140D0F0E75
:105B7800F324D96E010EF420DA6EDECFE6F0DDCF25
:105B8800E7F0E6510101B26FB36BFA93AD6BAE6B00
:105B980062D0E669E769ABC1E8F0ACC1E9F0E6516B
:105BA800E827E751E9230101AD510001E8190AE1AD
:105BB8000101AE510001E91905E10101B251B3112A
:105BC80001E1FA835050200D000EF3240001846F88
:105BD800020EF420856F340E866F0A0E876F010E51
:105BE800896F886BB40E8A6F010E8B6FFEEC11F013
:105BF8000101AF6FAF5101E025D7B4C148F0B5C17D
:105C080049F092EC32F05050140D070EF324D96E7F
:105C1800010EF420DA6E000EDE240001E66F010E9C
:105C2800DE20E76F000EDE20E86F000EDE20E96F51
:105C38005050140D070EF324D96E010EF420DA6EBD
:105C4800E6C0DEFFE7C0DEFFE8C0DEFFE9C0DEFF3A
:105C58000101AD4BAE2BAB51AD5DAE51800A0001D9
:105C6800E66F0101AC51800A0001E65992E3010197
:105C7800B3BF4CD0B35102E1B20548E35050200DF8
:105C8800000EF3240001846F020EF420856F340E99
:105C9800866F0A0E876FB2C188F0B3C189F0B40E5F
:105CA8008A6F010E8B6FFEEC11F00101AF6FAF51DF
:105CB80001E0C8D6FA83B2C148F0B3C149F092EC0A
:105CC80032F05050140D070EF324D96E010EF42053
:105CD800DA6E000EDE240001E66F010EDE20E76FAB
:105CE800000EDE20E86F000EDE20E96F5050140D24
:105CF800070EF324D96E010EF420DA6EE6C0DEFF3B
:105D0800E7C0DEFFE8C0DEFFE9C0DEFF0101FA936D
:105D18004E6A8390839E08D71550D96EDA6ADECF13
:105D280022F0DDCF23F002D0224A232A22C0F6FF38
:105D380023C0F7FF000EF86E0E0EF76403D00800BC
:105D4800F55005D0F6CFE9FFF7CFEAFFEF502F0A5D
:105D5800EBE022C0F6FF23C0F7FF000EF86E0E0E30
:105D6800F76403D00800F55005D0F6CFE9FFF7CF68
:105D7800EAFFEF505C0AD8E020EE14F01350D92661
:105D88001450DA22DECF24F0DDCF25F024C00BF04A
:105D980025C00CF00E6A200E0D6E106A0B0E0F6EE9
:105DA80016EC56F01E6A1EC026F0276A26C01CF0A4
:105DB80027C01DF0206A080E1F6E1C502224166E84
:105DC8001D502320176E16C0F6FF17C0F7FF000EF0
:105DD800F86E0E0EF76403D00800F55005D0F6CF24
:105DE800E9FFF7CFEAFFEF50286E1C4A1D2A200E64
:105DF8002864A7D02F0E281801E1A3D05C0E28181C
:105E080001E19FD02E0E281805E01F50265C205077
:105E1800275814E3080E1F182010D8A4060C2E0EBD
:105E2800281801E0060C276A080E266E206A0B0E59
:105E38001F6ED8901E36D8901E36BFD77F0E2864A6
:105E480002D0030E1E12800E286403D09F0E286411
:105E580006D0DF0E28644CD0FD0E286049D01C50B7
:105E68002224166E1D502320176E16C0F6FF17C089
:105E7800F7FF000EF86E0E0EF76403D00800F55019
:105E880005D0F6CFE9FFF7CFEAFFEF50216E1C4AA5
:105E98001D2A3F0E216403D07E0E216406D07F0E9A
:105EA8002164060CFD0E2160060C166817681FC0D9
:105EB80018F020C019F0165018261750192218503B
:105EC800265C1950275801E3060C26502424D96E65
:105ED80027502520DA6E28C0DFFF264A272A2650B9
:105EE8002424D96E27502520DA6E21C0DFFF26D062
:105EF8001C0E0B6EFE0E0C6E28C00DF00E6AA6EC82
:105F080054F00B500C1001E0060C400E286405D02C
:105F18005B0E286002D01E8209D0600E286406D06D
:105F28007B0E286003D01E80200E285E2650242475
:105F3800D96E27502520DA6E28C0DFFF264A272A87
:105F48003CD71C502224166E1D502320176E155066
:105F5800D96EDA6A16C0DEFF17C0DDFF200E28648E
:105F680003D01A6A1B6A03D01B6A040E1A6E1AC081
:105F780028F02650271001E1060C24C0D9FF25C0BF
:105F8800DAFFE50EDE1806E124C0D9FF25C0DAFFE6
:105F9800050EDF6E080E1F18201004E1D8901E367B
:105FA800D8901E361E50030BE80601E128881E50C3
:105FB8000C0B040A01E1288620EE0BF02450D926A8
:105FC8002550DA2228C0DFFF000C9151921193115D
:105FD800941128E120EE0AF08F51D9269051DA2247
:105FE800DECF9AF0DECF9BF0DECF9CF0DECF9DF0C7
:105FF8009A519B119C119D110FE020EE12F08F51C8
:10600800D9269051DA22DE509A5DDE509B59DE5037
:106018009C59DE509D5952E3010E9A6F9B6B9C6B05
:106028009D6B4CD08FC044F090C045F091C046F0B5
:1060380092C047F093C048F094C049F008EC1CF0B7
:1060480044C0A2F045C0A3F046C0A4F047C0A5F0E4
:106058000001A551A411A31109E1020EA25D06E2F7
:10606800010E8F6F906B916B926B000CA2290FE160
:10607800A3290DE1A4290BE1A52909E1A2C08FF00C
:10608800A3C090F0A4C091F0A5C092F0120020EE39
:1060980012F08F51D9269051DA22DE50A25DDE50DF
:1060A800A359DE50A459DE50A559E8E391C09AF0EF
:1060B80092C09BF093C09CF094C09DF09AC09EF053
:1060C8009BC09FF09CC0A0F09DC0A1F09E2B000E2D
:1060D8009F23A023A12320EE12F08F51D92690519F
:1060E800DA22DE509E5DDE509F59DE50A059DE5008
:1060F800A15911E3020E9E6F9F6BA06BA16B9D517E
:106108009C119B1108E1020E9A5D05E28F6B906B62
:10611800916B926B12008FC044F090C045F09EC006
:1061280046F09FC047F0A0C048F0A1C049F008EC75
:106138001CF044C0A2F045C0A3F046C0A4F047C07C
:10614800A5F00001A251A311A411A5111AE0A229DA
:1061580006E1A32904E1A42902E1A5298FE0A2050B
:10616800A311A411A5118AE09A519E19AFE19B5180
:106178009F19ACE19C51A019A9E19D51A119C6E054
:10618800A5D78FC060F090C061F09EC062F09FC03C
:1061980063F0A0C064F0A1C065F0666967696869CA
:1061A8000F0E696FABEC19F0996F99511CE1915181
:1061B80092119311941117E08FC060F090C061F0B4
:1061C80091C062F092C063F093C064F094C065F02F
:1061D8009EC066F09FC067F0A0C068F0A1C069F0DB
:1061E800ABEC19F0996F995130E120EE0AF08F511C
:1061F800D9269051DA229EC0DEFF9FC0DEFFA0C0E4
:10620800DEFFA1C0DEFF20EE0EF08F51D92690519F
:10621800DA22DE2806E1DE2804E1DE2802E1DE28B3
:1062280021E020EE0EF08F51D9269051DA22DE06B9
:10623800000EDE5ADE5ADE5A20EE05F08F51D926BE
:106248009051DA22000EDB800DD0990507E0010E8F
:106258009E6F000E9F6BA06BA16B04D09E699F6917
:10626800A069A1699EC08FF09FC090F0A0C091F076
:10627800A1C092F0120020EE04F08451D926855175
:10628800DA2286C0DEFF87C0DDFF20EE06F08451EB
:10629800D9268551DA22DECF95F0DECF96F0DECF13
:1062A80097F0DECF98F09505961197119811D8B40C
:1062B800020C84C0D9FF85C0DAFF10EE12F0DE5060
:1062C800E126DD50E222E650955DE6509659E6500B
:1062D8009759E650985901E3020C95519611971178
:1062E800981121E184C0D9FF85C0DAFFDECF88F09C
:1062F800DDCF89F088C0D9FF89C0DAFF030EDE1828
:1063080012E184C0D9FF85C0DAFF10EE22F0DE501A
:10631800E126DD50E222E6CF95F0E6CF96F0E6CF13
:1063280097F0E6CF98F0955196119711981123E1BF
:1063380084C0D9FF85C0DAFF10EE08F0DE50E126F0
:10634800DD50E222E650865DE650875901E3020CF3
:1063580084C0D9FF85C0DAFF10EE22F0DE50E126B6
:10636800DD50E222E6CF91F0E6CF92F0E6CF93F04F
:10637800E6CF94F074D084C0D9FF85C0DAFF10EE60
:1063880002F0DE50E126DD50E222E750100DF3CF97
:106398008FF0F4CF90F044D084C0D9FF85C0DAFFE5
:1063A800DECF44F0DDCF45F095C046F096C047F00B
:1063B80097C048F098C049F008EC1CF044C095F02C
:1063C80045C096F046C097F047C098F0000195295F
:1063D80007E1962905E1972903E1982901E1010CD4
:1063E80098519711961104E1020E955DD8A0020C00
:1063F80084C0D9FF85C0DAFF10EE12F0DE50E12626
:10640800DD50E222E650955DE6509659E6509759E0
:10641800E650985901E3020C8F51865F9051875BD3
:106428008F51865D90518759B7E284C0D9FF85C0E6
:10643800DAFFDECF0BF0DDCF0CF095C00DF096C083
:106448000EF097C00FF098C010F0F0EC45F00BC0BC
:1064580091F00CC092F00DC093F00EC094F00001C2
:1064680020EE0AF08451D9268551DA2295C0DEFF44
:1064780096C0DEFF97C0DEFF98C0DEFF91519211F3
:106488009311941101E1020C86C088F087C089F04D
:10649800040E8A6FD890893388338A2FFBD78851A6
:1064A80091258B6F895192218C6F000E93218D6FEE
:1064B800000E94218E6F20EE0EF08451D92685515E
:1064C800DA228BC0DEFF8CC0DEFF8DC0DEFF8EC0FF
:1064D800DEFF0F0E8615886F896B050ED8908837FA
:1064E8008937E82EFBD784C0D9FF85C0DAFFDECF15
:1064F8008AF0DDCF8BF088518A2789518B232E0EA5
:106508008A27000E8B2320EE12F08451D92685515C
:10651800DA228AC0DEFF8BC0DDFF000C0101A06B10
:106528004B6A4C6A898689808982898489888B68C4
:106538008490849284948498010EFCEC56F083B481
:106548000DD00101EEA707D0A10E0001606FFB0E70
:10655800616FE0EC56F0486A496A12000F01139126
:10656800350EE82EFED700F004D18EB813D0FB51BB
:1065780011E14CBE0FD04C5002E14B040BE3760EF8
:106588000001606FFE0E616FE0EC56F0630E0101D2
:10659800A06FF5D0100E786F270E796F7A6B7B6B32
:1065A800CFD08EB28EA411D001017807000E795B8E
:1065B8007A5B7B5B782906E1792904E17A2902E193
:1065C8007B29D8A4D6D0620E02D0010E5AD0A06F73
:1065D800D0D08EA8CED0020E54D08669876948C024
:1065E80088F049C089F086518827875189234B5004
:1065F800881906E14C50891903E10101FAB3899A17
:10660800340E4B24D96E0A0E4C20DA6EDF1C866ECF
:106618004B4A4C2A8B6A030E0101A06F100E786F4B
:10662800270E796F7A6B7B6B06D08EA204D0899087
:10663800050EA06F0FD07807000E795B7A5B7B5B45
:106648007829F3E17929F1E17A29EFE17B2901E160
:1066580090D0EBD7100E786F270E796F7A6B7B6B23
:1066680012D08EA410D0898A89808B6848504B5CE0
:106678004C50800A0001866F4950800A8659ABE366
:10668800630E0101A4D77807000E795B7A5B7B5B08
:106698007829E7E17929E5E17A29E3E17B2969E0CD
:1066A800E0D78EB20ED001017807000E795B7A5BD5
:1066B8007B5B782909E1792907E17A2905E17B29BA
:1066C80003E1040E0101A06F8EA253D0040E7FD700
:1066D8008990050E0101A06F100E786F270E796F53
:1066E8007A6B7B6B46D089848EB40ED00101780713
:1066F800000E795B7A5B7B5B782909E1792907E1F0
:106708007A2905E17B2903E1060E0101A06F8EA419
:1067180030D0060E5CD7898A89808B6848504B5CDC
:106728004C50800A866F4950800A865901E24DD73D
:10673800A7D79D0E606FFF0E616FE0EC56F0A0D7F3
:10674800A0510001866F876B875113E1865101E1E3
:1067580028D7010A01E13DD7030A01E13ED7010A22
:10676800A0E0070AB5E0010ABEE0030AD4E0640A23
:10677800E0E0630E0101A01902E08EBCF6D6898024
:10678800898289848988898A8B680F0113814BC023
:1067980048F04CC049F01200340E0101B76F0A0EE0
:1067A800B86FEDC00BF0EEC00CF0D0EC53F00B500E
:1067B8000101AB6FCD0E0001A66FA76BA86BA96B8B
:1067C800AA6BAB6B14EC0FF00101B46FB4510DE080
:1067D800580E0001606FFC0E616FE0EC56F000018E
:1067E800CD6BCE6BCF6BD06B1200CD0E0001846FDA
:1067F800856BB7C186F0B8C187F0010E896F886BC9
:10680800B20E8A6F010E8B6FFEEC11F00101B46FAE
:10681800B45108E0B80E0001606FFC0E616FE0EC47
:1068280056F0DDD7B7C1D9FFB8C1DAFF800EDE1840
:1068380008E05A0E0001606FFD0E616FE0EC56F043
:10684800CED720EE0AF0B751D926B851DA22DF5058
:106858000001F06FEF6B010120EE0BF0B751D92664
:10686800B851DA22DF500001EF250101B06F000EA8
:106878000001F0210101B16FA10E0001606FFC0E53
:10688800616FB0C162F0B1C163F0E0EC56F0CD0EBB
:106898000001A66FA76B0101B0510001F06FEF6B0B
:1068A800EFC0A8F0F0C0A9F0AA6BAB6B14EC0FF026
:1068B8000101B46FB45193E1CD0E0001846F856B73
:1068C800B7C186F0B8C187F0010E896F886BB20E28
:1068D8008A6F010E8B6FFEEC11F00101B46FB45199
:1068E80001E07DD7B56BB66BEDC00BF0EEC00CF0D8
:1068F800B5C1EFF0B6C1F0F0050ED8900001EF3742
:10690800F037E82EFAD7EF510101B7250D6E0001D7
:10691800F0510101B8210E6EABC10FF0106A21ECE5
:106928004DF00B500C105DE1B5C1EFF0B6C1F0F0C1
:10693800050ED8900001EF37F037E82EFAD7B7C127
:10694800F1F0B8C1F2F0EF51F127F051F2230E0E39
:10695800F125D96E000EF221DA6EDF50F46FF36B79
:10696800B5C1F5F0B6C1F6F0050ED890F537F63793
:10697800E82EFBD7B7C1F7F0B8C1F8F0F551F72703
:10698800F651F8230F0EF725D96E000EF821DA6EAE
:10699800DF50F96FFA6BF351F927F451FA23F9C074
:1069A800ACF1FAC0ADF10101000EADBFFF0EAE6F44
:1069B800AF6FFE0E0001606FFD0E616FACC162F03B
:1069C800ADC163F0AEC164F0AFC165F0E0EC56F064
:1069D800ACC1CDF0ADC1CEF0AEC1CFF0AFC1D0F0FB
:1069E8001200B54BB62BB6BF7FD7B65105E10F0ED7
:1069F800B55D01E3F4D678D7F2D646C00CF047C0AF
:106A08000DF068EC4DF000016C6F6C5101E000D1A5
:106A180020EE04F04650D9264750DA22DFAAF8D0F3
:106A280046C0D9FF47C0DAFFDECF39F0DDCF3AF0F4
:106A380020EE1AF04650D9264750DA22DECF3BF036
:106A4800DECF3CF0DECF3DF0DECF3EF0F5EC4BF094
:106A580000016C6F6C5101E0DBD020EE1EF0465057
:106A6800D9264750DA22DECF71F0DDCF72F020EE62
:106A78000BF07151D9267251DA22000EDB8A20EE12
:106A88000AF04650D9264750DA2210EE1CF0715110
:106A9800E1267251E222DFCFE7FF20EE1DF07151AF
:106AA800D9267251DA2210EE0AF04650E1264750F4
:106AB800E222E6CF68F0E5CF69F069C068F0696B5B
:106AC8006851DF6E20EE1EF07151D9267251DA221C
:106AD80010EE0AF04650E1264750E222E6CF68F071
:106AE800E6CF69F0E6CF6AF0E6CF6BF0110E05D07D
:106AF800D8906B336A3369336833E82EF9D7685115
:106B0800DF6E20EE1FF07151D9267251DA2210EE95
:106B18000AF04650E1264750E222E6CF68F0E6CF79
:106B280069F0E6CF6AF0E6CF6BF0190E05D0D89081
:106B38006B336A3369336833E82EF9D76851DF6EEF
:106B480071C00BF072C00CF020EE0EF04650D92642
:106B58004750DA22DECF0DF0DECF0EF0DECF0FF099
:106B6800DECF10F0AFEC53F000016D6B6E6B210EB1
:106B78006F6F460E706F20EE16F07151D926725164
:106B8800DA22DF6A20EE17F07151D9267251DA2223
:106B98006EC0DFFF20EE18F07151D9267251DA224B
:106BA8006FC0DFFF20EE19F07151D9267251DA2239
:106BB80070C0DFFF20EE12F07151D9267251DA222F
:106BC800DF6A20EE13F07151D9267251DA22DF6A9A
:106BD80020EE04F04650D9264750DA22DF0EDF16A1
:106BE80046C0D9FF47C0DAFF10EE04F0DE50E126B8
:106BF800DD50E222010EE76E46C0D9FF47C0DAFF3A
:106C0800DECF43F0DDCF44F07FEC2BF000016C6F5A
:106C18006C51120020EE04F04450D9264550DA2277
:106C2800DF6A20EE2AF04450D9264550DA22DE6881
:106C3800DE68DE68DD6844C039F045C03AF046C019
:106C48003BF047C03CF048C03DF049C03EF0F5EC91
:106C58004BF0000901E0030C22EE2DF04450D92638
:106C68004550DA22DF500001616F606B22EE2CF094
:106C78004450D9264550DA22DF506013550E60196A
:106C880003E1AA0E611901E0020C20EE65F0445000
:106C9800D9264550DA22DF50616F606B20EE66F02E
:106CA8004450D9264550DA22DF50626F62C063F043
:106CB800646B656B666B64C066F063C065F0646B9B
:106CC800636B20EE67F04450D9264550DA22DF5036
:106CD800676F67C068F0696B6A6B6B6B68C06BF055
:106CE8006A6B696B686B635168116C6F64516911E9
:106CF8006D6F65516A116E6F66516B116F6F6051E0
:106D08006C11706F61516D11716F000E6E11726FA1
:106D1800000E6F11736F20EE64F04450D926455071
:106D2800DA22DF507011746F7151756F7251766F7E
:106D38007351776F7451786F7551796F76517A6F97
:106D48007B6B460E781908E1410E791905E1540E5E
:106D58007A197B1101E1000C20EE81F04450D9260C
:106D68004550DA22DF50616F606B20EE82F04450AC
:106D7800D9264550DA22DF50626F62C063F0646B37
:106D8800656B666B64C066F063C065F0646B636BCB
:106D980020EE83F04450D9264550DA22DF50676F41
:106DA80067C068F0696B6A6B6B6B68C06BF06A6B85
:106DB800696B686B635168116C6F645169116D6F11
:106DC80065516A116E6F66516B116F6F60516C116E
:106DD800706F61516D11716F000E6E11726F000E40
:106DE8006F11736F20EE80F04450D9264550DA2297
:106DF800DF507011746F7151756F7251766F7351E6
:106E0800776F7451786F7551796F76517A6F7B6BA4
:106E1800460E781908E1410E791905E1540E7A19E0
:106E28007B1101E1000C010CC76B0101A16B030E82
:106E3800ED6105D09650ED19F00BED1905D0EDC1B7
:106E480093FF9650F00B0A09966ECD6ACE6ADFD092
:106E5800C86B340E156E0A0E166E220E176EFB0ED8
:106E6800186E59EC4BF015C0C5F016C0C6F0C5C079
:106E7800D9FFC6C0DAFF3B0EDE1801E0C3D0C7D089
:106E8800C85109E1C5C00FF0C6C010F0A7EC4FF01B
:106E98000001C76FA9D0C80511E10101F95100012E
:106EA800C71903E07F0EC71909E1C5C00FF0C6C0B6
:106EB80010F0A7EC4FF001019E6F96D0020EC81992
:106EC80011E10101F9510001C71903E07F0EC7194B
:106ED80009E1C5C00FF0C6C010F0A7EC4FF00101E2
:106EE8009D6F82D0020EC8651FD0080EC8611CD0E5
:106EF8000101F9510001C71903E07F0EC71914E118
:106F0800EF0EC36F010EC46FC5C00FF0C6C010F0FE
:106F1800A7EC4FF00001C06FC851C325C16F000E28
:106F2800C421C26FFD0E40D0070EC8651FD01B0ECE
:106F3800C8611CD00101F9510001C71903E07F0E97
:106F4800C71914E1A00EC36F020EC46FC5C00FF0BD
:106F5800C6C010F0A7EC4FF00001C06FC851C325A0
:106F6800C16F000EC421C26FF80E1ED0280EC86172
:106F780023D00101F9510001C71903E07F0EC71999
:106F88001BE1C60EC36F020EC46FC5C00FF0C6C0AA
:106F980010F0A7EC4FF00001C06FC851C325C16FB6
:106FA800000EC421C26FE50EC125D96EFF0EC221A5
:106FB800DA6EC0C0DFFF18D0280EC81915E101012C
:106FC800F9510001C71903E07F0EC7190DE1A10EA1
:106FD8000B6E010E0C6EC5C00DF0C6C00EF0106A27
:106FE800080E0F6E96EC51F00001C82B156A166A50
:106FF800220E176EFB0E186E59EC4BF015C0C5F03B
:1070080016C0C6F00001C551C61101E039D7340ECB
:107018000001AC6F0A0EAD6FAF6B910EAE6F000E34
:10702800B06F020EB16FA7EC4BF0AC51AD1101E09F
:107038000FD71200838E83804E6A89EC3EF0CDC054
:10704800B3F1CEC0B4F10101B351B41105E0B3C13D
:10705800EDF0B4C1EEF01200536AAB6BAC6BAD6BE4
:10706800AE6BB26B010EB16FB76BD2D0B56BB66BAE
:107078001CD078EC56F00B500C1013E0B70E0B6ECA
:10708800010E0C6EAFEC4DF00101B06F000E5324F1
:10709800D96EDA6A030EDA22B0C1DFFF532AB54B84
:1070A800B62B0101B7AB8EAC04D0B6BFE2D7B6059C
:1070B800E0E3B5C1EFF0B6C1F0F0000E0001F0BF9B
:1070C800FF0EF16FF26FEF510101AB270001F05194
:1070D8000101AC230001F1510101AD230001F2517E
:1070E8000101AE235050140D0F0EF324D96E010E7A
:1070F800F420DA6EDE50AB5DDE50AC59DE50AD598F
:10710800DE50AE5902E3B16BB26BB7AB02D0B16BD4
:10711800B26B8EBC02D0B16BB26BB6BF02D0B605F3
:1071280019E2000E53240B6E0C6A030E0C22FF0E9C
:107138005324D96EDA6A020EDA22DF500D6E0E6A17
:10714800535000080F6E000ED8A0E82A0108106EF0
:1071580092EC42F0010199513AE05050140D070E9B
:10716800F324D96E010EF420DA6E74C1F4F075C1FF
:10717800F5F076C1F6F00001F36B000EF325F76F1A
:10718800010EF421F86F000EF521F96F000EF621BB
:10719800FA6FDE50F7191BE1DE50F81918E1DE50DE
:1071A800F91915E1DE50FA1912E101C3BBF103C365
:1071B800BAF105C3B9F107C3B8F1B8C10EF0B9C146
:1071C8000FF0BAC110F0BBC111F015EC52F00BEC86
:1071D80051F0E4510101AF6FAF511AE0010E4E6E4C
:1071E8005050140D130EF324D96E010EF420DA6EEC
:1071F8005050140D130EF324E16E010EF420E26ECC
:10720800E7500409DF6E4EC0EDF00001EE6B12008E
:10721800B151B21101E02AD78FA402D0010E4E6EEF
:107228008390839E0001ED6BEE6B1200506A506AEA
:10723800030E506401D0E9D0505003E1486A496A0E
:1072480003D0496A010E486E5050140D130EF324F2
:10725800D96E010EF420DA6EDF6A5050140D000E5C
:10726800F324D96E010EF420DA6EDF6A5050140D43
:10727800070EF324D96E010EF420DA6EDE6ADE6A98
:10728800DE6ADD6A0D0E4802F3CF86F0F4CF87F090
:107298004902F35000018727D10E8625D96E020EC8
:1072A8008721DA6EDF50886F88C089F08A6B8B6B14
:1072B8008C6B8BC08CF08AC08BF089C08AF0896B8C
:1072C8000D0E4802F3CF8DF0F4CF8EF04902F35043
:1072D8008E27D00E8D25D96E020E8E21DA6EDF50E4
:1072E8008F6F8FC090F0916B926B936B91C093F0FE
:1072F80090C092F0916B906B0D0E4802F3CF94F012
:10730800F4CF95F04902F3509527CF0E9425D96E06
:10731800020E9521DA6EDF50966F96C097F0986B43
:10732800996B9A6B97C09AF0996B986B976B0D0E47
:107338004802F3CF9BF0F4CF9CF04902F3509C270E
:10734800CE0E9B25D96E020E9C21DA6EDF50972552
:107358009D6F000E98219E6F000E99219F6F000E61
:107368009A21A06F90519D25A16F91519E21A26FE6
:1073780092519F21A36F9351A021A46F8951A125F8
:10738800A56F8A51A221A66F8B51A321A76F8C519B
:10739800A421A86F5050140D0B0EF324D96E010EC2
:1073A800F420DA6EA5C0DEFFA6C0DEFFA7C0DEFFB0
:1073B800A8C0DEFFC60E606FFB0E616F50C062F0A2
:1073C800636B5050140D0B0EF324D96E010EF4208C
:1073D800DA6EDECF64F0DECF65F0DECF66F0DECFAA
:1073E80067F05050140D0B0EF324D96E010EF420E3
:1073F800DA6EDECF68F0DECF69F0DECF6AF0DECF7E
:107408006BF0E0EC56F0502A13D70101976B4F6AE6
:10741800966B886B896B020E4E6E8390020CFA8312
:10742800340E0B6E0A0E0C6E0E6A0D6A010E106E8B
:107438000F6A92EC42F02AEE34F050C0DFFFFF0EE4
:10744800E8CF35FA5050140D130EF324D96E010EFF
:10745800F420DA6EDFA403D0010EE8CF38FA5050DA
:10746800140D130EF324D96E010EF420DA6EDFA08A
:1074780003D0020EE8CF3AFA5050140D130EF3243D
:10748800D96E010EF420DA6EDFA203D0020EE8CF27
:107498003AFA5050140D130EF324D96E010EF4204D
:1074A800DA6EDFA603D0800EE8CF39FA8FA403D0B6
:1074B800080EE8CF3AFA00018B6B8C6BE60E606F12
:1074C800FB0E616FCECF62F0636BCDCF64F0656B5E
:1074D8008BC066F08CC067F0360E8B25D96E0A0E0D
:1074E8008C21DA6EDF50686F696BE0EC56F06C0E39
:1074F80000018B25D96E010E8C21DA6EDF1C8A6F94
:10750800360E8B25D96E0A0E8C21DA6E360E8B2537
:10751800E16E0A0E8C21E26EE7508A15DF6E5C0E72
:10752800606FFF0E616F360E8B25D96E0A0E8C21A7
:10753800DA6EDF50626F636BE0EC56F000018B4B44
:107548008C2B8CBFBBD78C5103E1070E8B5DB6E348
:107558005050140D130EF324D96E010EF420DA6E78
:10756800DF504E6E5050140D010EF324D96E010EEB
:10757800F420DA6EDF504A6E4AC03FFA5050140DBC
:10758800020EF324D96E010EF420DA6EDF504A6E33
:107598004AC040FA5050140D030EF324D96E010E60
:1075A800F420DA6EDF504A6E4AC041FA5050140D8A
:1075B800040EF324D96E010EF420DA6EDF504A6E01
:1075C8004AC042FA5050140D050EF324D96E010E2C
:1075D800F420DA6EDF504A6E4AC043FA5050140D58
:1075E800060EF324D96E010EF420DA6EDF504A6ECF
:1075F8004AC044FA496A140E486E92EC32F001010E
:10760800FA93839012008EA605D0370E0001866F7C
:10761800FE0E04D0B20E0001866FFF0E876F8EAA91
:1076280004D0370E886FFE0E03D0AD0E886FFF0EA4
:10763800896F8EA804D0370E8A6FFE0E03D0B70E5E
:107648008A6FFF0E8B6F8EAE04D0370E8C6FFE0ED6
:1076580003D0BC0E8C6FFF0E8D6F8EAC04D0370E2E
:107668008E6FFE0E03D0A80E8E6FFF0E8F6F8EA446
:1076780004D0370E906FFE0E03D0C60E906FFF0E2B
:10768800916F8EA204D0370E926FFE0E03D0CB0EF0
:10769800926FFF0E936F8EA004D0370E946FFE0E7C
:1076A80003D0C10E946FFF0E956F90AE04D0370EC5
:1076B800966FFE0E03D0F90E966FFF0E976F90AC83
:1076C80004D0370E986FFE0E03D0F60E986FFF0E9B
:1076D800996F90AA04D0370E9A6FFE0E03D0F30E5E
:1076E8009A6FFF0E9B6F90A804D0370E9C6FFE0E0A
:1076F80003D0F00E9C6FFF0E9D6F90A604D0370E3E
:107708009E6FFE0E03D0ED0E9E6FFF0E9F6F90A42E
:1077180004D0370EA06FFE0E03D0EA0EA06FFF0E46
:10772800A16F90A204D0370EA26FFE0E03D0E70E11
:10773800A26FFF0EA36F90A004D0370EA46FFE0EA9
:1077480003D0E40EA46FFF0EA56F240E606FFB0E2E
:10775800616F901C626F636B8ECF64F0656BA4C021
:1077680066F0A5C067F0A2C068F0A3C069F0A0C029
:107778006AF0A1C06BF09EC06CF09FC06DF09CC019
:107788006EF09DC06FF09AC070F09BC071F098C009
:1077980072F099C073F096C074F097C075F094C0F9
:1077A80076F095C077F092C078F093C079F090C0E9
:1077B8007AF091C07BF08EC07CF08FC07DF08CC0D9
:1077C8007EF08DC07FF08AC080F08BC081F088C0C9
:1077D80082F089C083F086C084F087C085F0E0EF2E
:1077E80056F05050070D520EF324D96E010EF420B6
:1077F800DA6EDF2A5050070D520EF324D96E010EAF
:10780800F420DA6E0F0EDF642FD05050070D520EA1
:10781800F324D96E010EF420DA6EDF6A5050070D9A
:10782800510EF324D96E010EF420DA6EDF2A50507F
:10783800070D510EF324D96E010EF420DA6E010EF5
:10784800DF6412D05050070D510EF324D96E010E8B
:10785800F420DA6EDF6A5050070D500EF324D96E0B
:10786800010EF420DA6EDF2A5050070D520EF32471
:10787800D96E010EF420DA6EDF500001CD6FCDC055
:10788800CEF0CF6BD06BD16BD0C0D1F0CFC0D0F0E1
:10789800CEC0CFF0CE6B5050070D510EF324D96EE9
:1078A800010EF420DA6EDF50D26FD2C0D3F0D46B61
:1078B800D56BD66B0C0ED890D337D437D537D6378F
:1078C800E82EF9D75050070D500EF324D96E010E4B
:1078D800F420DA6EDF50D76FD7C0D8F0D96BDA6BE7
:1078E800DB6B0D0ED890D837D937DA37DB37E82E6F
:1078F800F9D7D351D825DC6FD451D921DD6FD551B3
:10790800DA21DE6FD651DB21DF6FCE51DC25E06F47
:10791800CF51DD21E16FD051DE21E26FD151DF215E
:10792800E36F5050070D530EF324D96E010EF42067
:10793800DA6EE0C0DEFFE1C0DEFFE2C0DEFFE3C0DA
:10794800DEFF5050200D000EF324A66F020EF42027
:10795800A76F5050070D530EF324D96E010EF42073
:10796800DA6EDECFA8F0DECFA9F0DECFAAF0DECF48
:10797800ABF014EC0FF04A6E4A5019E0710E606FCC
:10798800FC0E616F5050070D530EF324D96E010E93
:10799800F420DA6EDECF62F0DECF63F0DECF64F083
:1079A800DECF65F04AC066F0676BE0EC56F0010187
:1079B800946B12000001AE6FAA5102E01AEC39F084
:1079C8000001AD6BA95101E1B9D0040EAE1903E075
:1079D800140EAE1909E10101966B886B896B0001E1
:1079E800AA6B070EA96F070C3F0EAE1907E14F6A85
:1079F8000101966B0001A96BAA6B12005F0EAE190C
:107A080007E10101976B966B0001A96BAA6B120045
:107A18003F0EAE6506D05F0EAE6103D0400EAE19C4
:107A2800F0E1400EAE1908E1010E0101976F966B67
:107A38000001A96BAA6B1200200EAE190CE1010E11
:107A48004F6E0101966B7F0E0001606FFF0E616F34
:107A5800E0EC56F0EDD7650EAE1909E14F5007E09E
:107A68000101886B896B010E966F8380E1D76E0EDA
:107A7800AE1903E1020E0101966F700E0001AE19F6
:107A880007E10101975104E0886B896B030E966F3B
:107A9800700E0001AE1908E14F5006E08380010125
:107AA800886B896B040E0CD0720EAE1947E14F50EB
:107AB80045E083801C0E0101896F2A0E886F050E30
:107AC800966FB6D7AE51B4EC14F00001AD6F49D043
:107AD8008380AE517AEC4EF00001AD6F0101966BD8
:107AE80040D08380340E0B6E0A0E0C6E0E6A0D6A3F
:107AF800010E106E0F6A92EC42F00101FA832AEE31
:107B080034F04EC0DFFF496A010E486E92EC32F045
:107B18000101FA93080EE0D78390AD6B22D0080ECE
:107B2800AE1901E103D0090EAE191BE18390AD6BCC
:107B38004E6A0101966B886B896B13D001019651CF
:107B48000001AB6FAC6BAC510CE1AB510AE0010A20
:107B5800B9E0030ABDE0010AC4E0070ADDE0010A52
:107B6800DEE0ADC0A9F00001AA6B12000001BD6BF8
:107B7800010EBC6F838E8380BED05050200D000E46
:107B8800F324846F020EF420856F340E866F0A0E7C
:107B9800876F010E896F886BBE0E8A6F8B6BFEEC48
:107BA80011F0010199514BE05050070D530EF32489
:107BB800D96E010EF420DA6E74C1B1F075C1B2F05D
:107BC80076C1B3F00001B06B000EB025B46F010EA2
:107BD800B121B56F000EB221B66F000EB321B76F99
:107BE800DE50B4192CE1DE50B51929E1DE50B61982
:107BF80026E1DE50B71923E116EC50F00FC0C0F0B3
:107C080010C0C1F011C0C2F012C0C3F0000EE8CF1E
:107C180034FA2AEE35F0C3C0DFFFE8CF36FA2AEE91
:107C280037F0C2C0DFFFE8CF38FA2AEE39F0C1C01A
:107C3800DFFFE8CF3AFA2AEE3BF0C0C0DFFF0101D0
:107C4800FA93BEC048F0BFC049F092EC32F048C089
:107C5800BAF049C0BBF08EAC53D00001BE51BA197E
:107C680003E1BF51BB190BE0AE0E606FFE0E616FF2
:107C7800BAC062F0BBC063F0E0EC56F041D097ECBC
:107C880056F078EC56F00B500C1004E0010E010190
:107C9800946F36D00001B96B050EB86F1CD0D00EAA
:107CA8000001AC6FC90EE82EFED7AC2FFCD700D070
:107CB80078EC56F00B500C100EE00001BC6BBD6B5D
:107CC8009E0E606FFD0E616FB8C062F0B9C063F0C0
:107CD800E0EC56F008D00001B807D8A0B907B829D9
:107CE800DEE1B929DCE178EC56F00B500C1003E02A
:107CF8000001BC6BBD6B0001BC51BD1101E03DD75B
:107D08000101946B839E839012005050140D070E4E
:107D1800F324D96E010EF420DA6EDECFDFF0DECF69
:107D2800E0F0DECFE1F0DECFE2F05050140D070EA8
:107D3800F324D96E010EF420DA6E5050140D0B0E98
:107D4800F324E16E010EF420E26EDE50E65CDE50B4
:107D5800E658DE50E658DE50E65815E2010E4E6E43
:107D68005050140D130EF324D96E010EF420DA6E60
:107D78005050140D130EF324E16E010EF420E26E40
:107D8800E7500409DF6E5050140D0F0EF324D96E1E
:107D9800010EF420DA6EDECFCFF0DECFD0F0DECFEA
:107DA800D1F0DECFD2F05050140D070EF324D96E67
:107DB800010EF420DA6EDECFD3F0DECFD4F0DECFC2
:107DC800D5F0DECFD6F00001CF51D325D76FD051F3
:107DD800D421D86FD151D521D96FD251D621DA6F9C
:107DE8005050140D0B0EF324D96E010EF420DA6EE8
:107DF800D751DE5CD851DE58D951DE58DA51DE58F9
:107E080015E2010E4E6E5050140D130EF324D96E68
:107E1800010EF420DA6E5050140D130EF324E16EA7
:107E2800010EF420E26EE7500409DF6E4E6A5050EE
:107E3800200D000EF324A66F020EF420A76FDFC0FA
:107E4800A8F0E0C0A9F0E1C0AAF0E2C0ABF014ECE1
:107E58000FF0E36FE35115E0010E4E6E5050140D14
:107E6800130EF324D96E010EF420DA6E5050140D5F
:107E7800130EF324E16E010EF420E26EE7500409BC
:107E8800DF6E4EC0CDF0CE6B12001B6E1B5001E0B2
:107E9800010C54A202D054501200000E40EC56F0CF
:107EA8000A0E266E03D004EC57F026062650FBE196
:107EB800236A000E146A156A166A176AC2EC54F02F
:107EC800E80601E097D0AA0E146E010E156E166A28
:107ED800176A080EC2EC54F0E80651E1266A2650EB
:107EE8001C0FD96EDA6A04EC57F0DF6E262A030EEF
:107EF8002664F5D71E047EE1AA0E1F187BE1030E47
:107F0800256EE80E246E15D0146A156A166A400E9E
:107F1800176EA90EC2EC54F000090EE0150E1A6E89
:107F2800C60EE82EFED71A2EFCD700D02406D8A0FD
:107F3800250624502510E8E1245025105BE0146A3A
:107F4800156A166A176A3A0EC2EC54F0000952E133
:107F5800266A26501C0FD96EDA6A04EC57F0DF6ED9
:107F6800262A030E2664F5D71CBC03D0216A040E0A
:107F780002D0216A0C0E206E20C023F03BD0146A78
:107F8800156A166A176AA90EC2EC54F01A6E020E28
:107F98001A6003D0236EA90E02D0010E236E226E42
:107FA800030E256EE80E246E14D0146A156A166A3C
:107FB800176A2250C2EC54F000090EE0150E1A6E32
:107FC800C60EE82EFED71A2EFCD700D02406D8A05D
:107FD800250624502510E9E1245025100AE0146AEA
:107FE800020E156E166A176A100EC2EC54F00009DC
:107FF80001E0236A23C051F01BEC57F0235001E144
:108008004AD7549048D7C1C0F6FFC2C0F7FF000E48
:10801800F86E0E0EF76403D00800F55005D0F6CFC1
:10802800E9FFF7CFEAFFEF502F0A13E0C1C0F6FFD0
:10803800C2C0F7FF000EF86E0E0EF76403D00800FA
:10804800F55005D0F6CFE9FFF7CFEAFFEF505C0A0D
:1080580003E10001C14BC22B000120EE06F0BF5125
:10806800D926C051DA22DE6ADE6ADE6ADD6AC1C05C
:10807800F6FFC2C0F7FF000EF86E0E0EF76403D0CD
:108088000800F55005D0F6CFE9FFF7CFEAFFEF502B
:108098004A6E200E4A6013D0BFC084F0C0C085F07D
:1080A8000001876B866B3FEC31F0C66F20EE12F053
:1080B800BF51D926C051DA22DE6ADD6A5DD0BFC061
:1080C80013F0C0C014F0C10E156E90EC2EF0000134
:1080D800C66FC65151E1BFC0B9F0C0C0BAF0C7EC15
:1080E80048F0C66F20EE14F0BF51D926C051DA22ED
:1080F80010EE0BF0DE50E126DD50E222E750C56FAE
:10810800C65108E0040EC61937E1C5B535D0050ECD
:10811800C66F32D0C5B530D020EE12F0BF51D92687
:10812800C051DA22DECFC3F0DDCFC4F020EE0BF071
:10813800C351D926C451DA22DFA8E9D7BFC0D9FF75
:10814800C0C0DAFFDECF0BF0DDCF0CF0C3C00DF0FE
:10815800C4C00EF0B2EC4AF0000120EE06F0BF51A8
:10816800D926C051DA220BC0DEFF0CC0DEFF0DC0DD
:10817800DEFF0EC0DEFFA3D7C6511200326A20EE22
:1081880004F02450D9262550DA22DF5001E197D097
:1081980020EE2AF02450D9262550DA22DECF35F0F9
:1081A800DECF36F0DECF37F0DECF38F02E0E2424C7
:1081B8001A6E000E25201B6E35C01CF036C01DF04F
:1081C80037C01EF038C01FF0216A010E206E20EE65
:1081D80001F02450D9262550DA22DF50E9EC47F087
:1081E800000903E0010E326E6AD020EE04F024503C
:1081F800D9262550DA22DF6A20EE16F02450D92637
:108208002550DA2210EE1EF02450E1262550E222F5
:10821800E6CF2AF0E6CF2BF0E6CF2CF0E6CF2DF014
:108228002A50355C2E6E2B5036582F6E2C503758EE
:10823800306E2D503858316EDE502E5CDE502F587F
:10824800DE503058DE5031583AE220EE03F0245028
:10825800D9262550DA22DF50336E346A345003E1D0
:10826800020E335C2CE320EE16F02450D92625505C
:10827800DA22DE503526DE503622DE503722DD5037
:1082880038222E0E24241A6E000E25201B6E35C0AF
:108298001CF036C01DF037C01EF038C01FF0216A30
:1082A800010E206E20EE01F02450D9262550DA2246
:1082B800DF50E9EC47F03306D8A03406CFD7325068
:1082C80012005050070D520EF324D96E010EF420FF
:1082D800DA6EDF500001CD6FCDC0CEF0CF6BD06B22
:1082E800D16BD0C0D1F0CFC0D0F0CEC0CFF0CE6B24
:1082F8005050070D510EF324D96E010EF420DA6E9A
:10830800DF50D26FD2C0D3F0D46BD56BD66B0C0EC6
:10831800D890D337D437D537D637E82EF9D7505039
:10832800070D500EF324D96E010EF420DA6EDF50DB
:10833800D76FD7C0D8F0D96BDA6BDB6B0D0ED8903E
:10834800D837D937DA37DB37E82EF9D7D351D825DC
:10835800DC6FD451D921DD6FD551DA21DE6FD651CA
:10836800DB21DF6FCE51DC25E16FCF51DD21E26FDC
:10837800D051DE21E36FD151DF21E46F5050200D41
:10838800000EF324A66F020EF420A76FE1C0A8F038
:10839800E2C0A9F0E3C0AAF0E4C0ABF014EC0FF01F
:1083A800E06FE05111E0710E606FFC0E616FE1C08B
:1083B80062F0E2C063F0E3C064F0E4C065F0E0C0DE
:1083C80066F0676BE0EC56F05050070D530EF3243F
:1083D800D96E010EF420DA6EE1C0DEFFE2C0DEFFE6
:1083E800E3C0DEFFE4C0DEFF0101946B839012005E
:1083F8002F6C696664617461302E62696E20002F8B
:108408006C696664617461312E62696E20002F6C3C
:10841800696664617461322E62696E20002F6C692E
:108428006664617461332E62696E20002F6C696620
:1084380064617461342E62696E20002F6C69666411
:10844800617461352E62696E20002F6C6966646103
:108458007461362E62696E20002F6C6966646174DF
:1084680061372E62696E20002F6C696664617461E1
:10847800382E62696E20002F6C69666461746139F8
:108488002E62696E20002F6C696664617461612ECA
:1084980062696E20002F6C696664617461622E6285
:1084A800696E20002F6C696664617461632E62696D
:1084B8006E20002F6C696664617461642E62696E57
:1084C80020002F6C696664617461652E62696E2094
:1084D800002F6C696664617461662E62696E2000A3
:1084E8000000000000000000000000000000000084
:1084F8000000000000000000000000000000000074
:108508000000000000000000000000000000000063
:108518000000000000000000000000000BC015F083
:108528000CC016F00F50101001E1120015C0D9FF51
:1085380016C0DAFF0DC0DFFF0F501524116E105062
:108548001620126EFF0E1124D96EFF0E1220DA6E5D
:108558000DC0DFFF105004E1030E0F5C01E21200B2
:1085680020EE01F01550D9261650DA220DC0DFFF93
:1085780020EE02F01550D9261650DA220DC0DFFF82
:108588000F501524116E10501620126EFE0E112475
:10859800D96EFF0E1220DA6E0DC0DFFF0F501524C2
:1085A800116E10501620126EFD0E1124D96EFF0E9A
:1085B8001220DA6E0DC0DFFF105004E1070E0F5CC9
:1085C80001E2120020EE03F01550D9261650DA22E7
:1085D8000DC0DFFF0F501524116E10501620126EBB
:1085E800FC0E1124D96EFF0E1220DA6E0DC0DFFFCB
:1085F800105004E1090E0F5C01E2120015C011F0E1
:1086080016C012F0111E121E114A122A030E11145E
:10861800136E146A135015261450162213500F5E49
:108628001450105AFC0E0F160BD015C0D9FF16C0E7
:10863800DAFF0DC0DFFF0F06D8A01006154A162A6C
:108648000F501010F2E11200000194519311921191
:1086580003E1020E915D0FE320EE12F08F51D9264F
:108668009051DA22DE50915DDE509259DE509359D6
:10867800DE50945902E3020E2CD0996B6AD08FC059
:1086880044F090C045F091C046F092C047F093C0C6
:1086980048F094C049F008EC1CF044C09AF045C07A
:1086A8009BF046C09CF047C09DF000019A519B1179
:1086B8009C119D115DE09A059B119C119D11DBE0B9
:1086C8009A2909E19B2907E19C2905E19D2903E1F4
:1086D800010E996F4DD08FC060F090C061F091C0CD
:1086E80062F092C063F093C064F094C065F0666B6A
:1086F800676B686B696BABEC19F0996F995138E14E
:1087080020EE0EF08F51D9269051DA22DE2806E1AC
:10871800DE2804E1DE2802E1DE2813E020EE0EF078
:108728008F51D9269051DA22DE2A000EDE22DE226F
:10873800DE2220EE05F08F51D9269051DA22000E64
:10874800DB809AC091F09BC092F09CC093F09DC0D2
:1087580094F020EE12F08F51D9269051DA22DE5093
:10876800915DDE509259DE509359DE50945987E35B
:1087780099511200136814680B50D96EDA6ADE50EA
:10878800DE1001E181D00B50D96EDA6ADECF17F026
:10879800DDCF18F002D0174A182A17C0F6FF18C004
:1087A800F7FF000EF86E0E0EF76403D00800F550C0
:1087B80005D0F6CFE9FFF7CFEAFFEF500D6E200E98
:1087C8000D6413D017C0F6FF18C0F7FF000EF86E3F
:1087D8000E0EF76403D00800F55005D0F6CFE9FF78
:1087E800F7CFEAFFEF503A0AD6E117C0F6FF18C0F4
:1087F800F7FF000EF86E0E0EF76403D00800F55070
:1088080005D0F6CFE9FFF7CFEAFFEF503A0A41E18A
:108818000B50D96EDA6ADECF11F0DDCF12F011C03D
:10882800F6FF12C0F7FF000EF86E0E0EF76403D0C5
:108838000800F55005D0F6CFE9FFF7CFEAFFEF5073
:108848000D6ED00E0D24156E166AFF0E1622114AF3
:10885800122A165019E10A0E155C16E21750111863
:1088680013E11850121810E1155016100DE115C03B
:1088780013F016C014F0174A182A0B50D96EDA6A8A
:1088880017C0DEFF18C0DDFF13C00BF014C00CF0DA
:108898001200136A146AF8D7838E83800001F16B83
:1088A800F26BADEC50F015C0F3F016C0F4F0000117
:1088B800F4BF0AD0040EF45D07E3000EF325F16F50
:1088C800FC0EF421F26F04D0F3C0F1F0F4C0F2F022
:1088D800010199513AE05050070D530EF324D96E17
:1088E800010EF420DA6E74C1E9F075C1EAF076C1C0
:1088F800EBF00001E86B000EE825EC6F010EE921B2
:10890800ED6F000EEA21EE6F000EEB21EF6FDE50E7
:10891800EC191BE1DE50ED1918E1DE50EE1915E1F6
:10892800DE50EF1912E101C3F8F003C3F7F005C3F5
:10893800F6F007C3F5F0F5C00EF0F6C00FF0F7C07B
:1089480010F0F8C011F015EC52F08FB415D050505B
:10895800200D000EF3240001A66F020EF420A76F6D
:10896800000EA86F030EA96F010EAB6FAA6BF10E74
:10897800AC6FA6EC0BF0F06F0001F05109E0AE0E01
:10898800606FFD0E616FF0C062F0636BE0EC56F053
:10899800F5EC3BF0946B8390839E490E0001606F69
:1089A800FD0E616FCECF62F0636BCDCF64F0656B67
:1089B800E0EF56F0F9C186F077D067EC56F0000189
:1089C800866F0101F951000186197CE0290E496E74
:1089D800960E486E7F0EE82EFED7482EFCD7492EFD
:1089E800FAD700F06FD0DFEC52F00001876F8751A3
:1089F80069E087B1522A87B352060F0E5216000E4D
:108A08000B6EC00E90EC52F02BEC56F0000E0B6E75
:108A1800C00E90EC52F052500F0D340EF3240F6E2E
:108A28000C0EF420106EBCEC4EF0110E496E3C0E8C
:108A3800486ECB0EE82EFED7482EFCD7492EFAD723
:108A480000F0000187A53ED00C6A0B6A52C00DF0F9
:108A580089EC54F0240E0001606FFD0E616F52C066
:108A680062F0636BE0EC56F052C086F0000E0B6EBD
:108A7800800E90EC52F02BEC56F0000E0B6E800E30
:108A880090EC52F052500F0D340EF3240F6E0C0E72
:108A9800F420106EBCEC4EF0000E0B6EC00E90EC85
:108AA80052F02BEC56F00ED001019B51486E496AEA
:108AB800495008E14850010A80E0030A01E17DD7E6
:108AC800010A91E0000186511200946B8380838E25
:108AD800000E0B6E030E0C6E0E6AF60E0D6E010E76
:108AE800106E0F6A92EC42F0850E0001606FFE0E68
:108AF800616FE0EC56F00001ED6BEE6BEDC0E5F058
:108B0800010EE517E533E5338350E5197F0BE519C9
:108B1800836E2E0ED5EC56F08FB415D05050200D24
:108B2800000EF3240001A66F020EF420A76F000EBA
:108B3800A86F030EA96F010EAB6FAA6BE70EAC6F9F
:108B4800A6EC0BF0E96F0001E95109E0630E606FD4
:108B5800FF0E616FE9C062F0636BE0EF56F078ECEE
:108B680056F00B500C1027E0EA0E0B6E0C6AAFECB7
:108B78004DF00001E66FEA51100B486E000E496E89
:108B8800E6513EEC22F048C0EBF049C0ECF0040E90
:108B98000001EB19EC1102E18FEC55F0020E000117
:108BA800EB19EC1102E1B8EC52F00001EB05EC1105
:108BB80002E165EC41F00001ED4BEE2B600EED5D3E
:108BC800040EEE599BE31D0E606FFF0E616FE0EC23
:108BD80056F0839E83901200020E0D5E000E0E5A10
:108BE8000F5A105A20EE12F00B50D9260C50DA22E8
:108BF800FE0EDE24116EFF0EDE20126EFF0EDE204A
:108C0800136EFF0EDE20146E11500D5C12500E58BC
:108C180013500F581450105805E30B6A0C6A0D6A6C
:108C28000E6A120020EE26F00B50D9260C50DA22DC
:108C3800DECF11F0DECF12F0DECF13F0DECF14F06E
:108C480020EE02F00B50D9260C50DA22DF50156EB8
:108C580015C016F0176A186A196A16500D02F3CF74
:108C68001AF0F4CF1BF01C6A1D6A0E02F3501B2683
:108C7800F4501C22000E1D2217500D02F3501B2623
:108C8800F4501C22000E1D2216500F02F3501C2611
:108C9800F4501D2217500E02F3501C26F4501D22CA
:108CA80018500D02F3501C26F4501D2210501602C5
:108CB800F3501D2617500F02F3501D2618500E02B0
:108CC800F3501D2619500D02F3501D2611501A2479
:108CD8000B6E12501B200C6E13501C200D6E14507E
:108CE8001D200E6E12001F6A206A186A196A01D0C8
:108CF800122A010E1E6E1250D96EDA6A200EDE1884
:108D080013E0F70E146E15681250D96EDA6ADF5048
:108D1800166E176A1450162615501722175003E1BD
:108D2800050E165C01E31E6A1EC01AF01B6A1A5073
:108D38001B1006E0DDD7196A010E186E122A25D01D
:108D48001250D96EDA6ADF50146E156A15501DE19B
:108D580014502B0AF3E0060AEEE017D00A0E1F02A1
:108D6800F3CF14F0F4CF15F02002F350152612506B
:108D7800D96EDA6ADF50145E000E155A300E1424CC
:108D88001F6E000E1520206ED9D7D00E146E1568F0
:108D98001250D96EDA6ADF50166E176A145016260A
:108DA80015501722175005E10A0E165C02E2010E53
:108DB80001D0000E1C6E1D6A1C501D10CFE118500A
:108DC80019100DE11FC014F020C015F0141E151E57
:108DD800144A152A14C012F015C013F012001FC04F
:108DE80012F020C013F012000001F26B8380838E12
:108DF80073D0ADEC50F015C0F0F016C0F1F00001E2
:108E0800F1BF06D0040EF15D03E3010EF26F03D04B
:108E1800F5C0F3F0F46B8FB414D05050200D000E51
:108E2800F324A66F020EF420A76F000EA86F030E9E
:108E3800A96F010EAB6FAA6BF30EAC6FA6EC0BF02B
:108E4800F56FF55109E0AE0E606FFD0E616FF5C06C
:108E580062F0636BE0EC56F0010199513AE0505032
:108E6800070D530EF324D96E010EF420DA6E74C187
:108E7800E9F075C1EAF076C1EBF00001E86B000E8D
:108E8800E825EC6F010EE921ED6F000EEA21EE6F87
:108E9800000EEB21EF6FDE50EC191BE1DE50ED19EF
:108EA80018E1DE50EE1915E1DE50EF1912E101C3A9
:108EB800F9F003C3F8F005C3F7F007C3F6F0F6C0FE
:108EC8000EF0F7C00FF0F8C010F0F9C011F015EC73
:108ED80052F0F5EC3BF0946B0001F2518AE0839E6E
:108EE800839012000F015969116B196B216B8C94D7
:108EF8008C928C90889A110E106E3C0E0F6ECB0ED1
:108F0800E82EFED70F2EFCD7102EFAD700F0110E40
:108F1800106E3C0E0F6ECB0EE82EFED70F2EFCD730
:108F2800102EFAD700F0020E106EA00E0F6E920EE1
:108F3800E82EFED70F2EFCD7102EFAD700D0000E41
:108F48000B6E300E90EC52F02A0E0F6E8E0EE82E3D
:108F5800FED70F2EFCD7000E0B6E300E90EC52F0A1
:108F6800000E0B6E300E90EC52F0000E0B6E390EA8
:108F780090EC52F0000E0B6E140E90EC52F0000EB6
:108F88000B6E560E90EC52F0000E0B6E6D0E90ECC0
:108F980052F0000E0B6E700E90EC52F0000E0B6E3D
:108FA8000C0E90EC52F0000E0B6E060E90EC52F088
:108FB800000E0B6E010E90EC52F0D00E0F6ECA0E22
:108FC800E82EFED70F2EFCD71200236E2350D8A40C
:108FD800040C2050211001E1040C54B0030C54B4CB
:108FE800020C51B608D0090ED8901C361D361E3614
:108FF8001F36E82EF9D7200421101AE11CC014F0FE
:109008001DC015F01EC016F01FC017F0180EC2ECD8
:1090180054F0000945E11AC00DF01BC00EF0FE0E19
:109028000F6EC1EC51F000093BE0206A216A38D08C
:1090380051C022F0060E221609E020C014F021C00B
:1090480015F0166A176A970EC2EC54F01CC014F09B
:109058001DC015F01EC016F01FC017F0190EC2EC87
:1090680054F000091DE11AC00DF01BC00EF0FC0EF3
:109078000F6EC1EC51F0000908E0020E1B26200615
:10908800D8A0210620502110EEE10D6A0E6AFD0ECF
:109098000F6EC1EC51F0000903E1216A010E206E48
:1090A8001BEC57F020502110D8A4010C000C818E25
:1090B800819CF80EF66E830EF76E000EF86E0CEEBD
:1090C80034F011EE2CF00900F5CFEEFFE550E15039
:1090D800FAE1E250F8E1E20EF66EA70EF76E000E26
:1090E800F86E02EEA0F010EE40F00900F5CFEEFFAA
:1090F800E550E150FAE1160EF66EAE0EF76E000E70
:10910800F86E01EEEDF010EE0CF00900F5CFEEFF71
:10911800E550E150FAE15A0EF66EAE0EF76E000E0B
:10912800F86E0900F5CF54F004EE00F018EE34F0B4
:10913800EE6AE550E150FCE1E250FAE103EE00F09E
:1091480011EE00F0EE6AE550E150FCE1E250FAE180
:1091580002EE00F0A00EEE6AE806FDE101EE00F076
:10916800AB0EEE6AE806FDE10001FF6B00EE4BF086
:10917800090EEE6AE806FDE155905592000EF86E6C
:109188000001F2EF07F0B9C084F0BAC085F0876B30
:10919800866B3FEC31F0BE6FBE5102E0BE5112004B
:1091A800B9C0D9FFBAC0DAFFDECF39F0DDCF3AF067
:1091B80020EE0EF0B951D926BA51DA22DECF3BF0B3
:1091C800DECF3CF0DECF3DF0DECF3EF0F5EC4BF0ED
:1091D8000001BE6FBE51E2E120EE12F0B951D9266E
:1091E800BA51DA22DECFBCF0DDCFBDF0BCC0D9FF6A
:1091F800BDC0DAFFDF50BB6FBB5103E1040EBE6F89
:10920800CDD720EE0BF0BC51D926BD51DA22DFB6FE
:1092180016D0BCC00BF0BDC00CF020EE14F0B95154
:10922800D926BA51DA22DECF0DF0DDCF0EF0106A62
:109238000B0E0F6E69EC51F00B500C10AFE0B9C07B
:10924800A6F0BAC0A7F0A96BA86B3CEC24F000010B
:10925800BE6FBE51A3E1A4D7B9C084F0BAC085F0EF
:10926800876B866B3FEC31F0C26FC25157E1C06B20
:10927800C16BB9C0D9FFBAC0DAFFDECF39F0DDCF94
:109288003AF020EE0EF0B951D926BA51DA22DECFE3
:109298003BF0DECF3CF0DECF3DF0DECF3EF0F5EC2C
:1092A8004BF00001C26FC25139E120EE12F0B95102
:1092B800D926BA51DA22DECFBDF0DDCFBEF0BDC06F
:1092C800D9FFBEC0DAFFE50EDE1810E020EE12F07E
:1092D800B951D926BA51DA22DECFBDF0DDCFBEF0C2
:1092E800BDC0D9FFBEC0DAFFDF5009E1C04BC12BBA
:1092F800BB51C01906E1BC51C11910E002D0C06BC6
:10930800C16BB9C0A6F0BAC0A7F0A96B010EA86FCF
:109318003CEC24F00001C26FC251ABE0040EC2194C
:1093280002E1070EC26FC2511200C3C0B9F0C4C037
:10933800BAF0BC6B010EBB6F30EC49F04A6E4A5074
:1093480053E1C3C0D9FFC4C0DAFFDECF39F0DDCFA7
:109358003AF020EE0EF0C351D926C451DA22DECFFE
:109368003BF0DECF3CF0DECF3DF0DECF3EF0F5EC5B
:109378004BF04A6E4A5038E1000120EE12F0C3511A
:10938800D926C451DA22DECF0BF0DDCF0CF00E6AFD
:109398000D6A106A200E0F6E16EC56F0000120EED2
:1093A80012F0C351D926C451DA22DECF0BF0DDCF3B
:1093B8000CF020EE14F0C351D926C451DA22DECFC6
:1093C8000DF0DDCF0EF0106A0B0E0F6E11EC54F09D
:1093D800C3C0D9FFC4C0DAFF10EE04F0DE50E126A6
:1093E800DD50E222010EE76E4A5012008380838E20
:1093F800000E0B6E030E0C6E0E6AF60E0D6E010E4D
:10940800106E0F6A92EC42F0850E0001606FFE0E3E
:10941800616FE0EC56F00001CC6BCD6BCCC04AF02C
:10942800010E4A164A324A3283504A187F0B4A18AC
:10943800836E2E0ED5EC56F08FB415D05050200DFB
:10944800000EF3240001A66F020EF420A76F000E91
:10945800A86F030EA96F010EAB6FAA6BC90EAC6F94
:10946800A6EC0BF0CB6F0001CB5109E0630E606FE7
:10947800FF0E616FCBC062F0636BE0EF56F0CC4B30
:10948800CD2BCDBFCBD7CD5103E1640ECC5DC6E368
:109498001D0E606FFF0E616FE0EC56F0839E8390A7
:1094A80083904E6A1200FA83505028E1340E0B6EF6
:1094B8000A0E0C6EEF0E0D6E010E0E6E106A050E82
:1094C8000F6E8EEC53F0390E0B6E0A0E0C6EA00E5A
:1094D8000D6E020E0E6E106A130E0F6E8EEC53F0A8
:1094E8004C0E0B6E0A0E0C6EC60E0D6E020E0E6E34
:1094F800106A0D0E0F6E8EEC53F027D0340E0B6EE3
:109508000A0E0C6EF40E0D6E010E0E6E106A050E2C
:109518000F6E8EEC53F0390E0B6E0A0E0C6EB30EF6
:109528000D6E020E0E6E106A130E0F6E8EEC53F057
:109538004C0E0B6E0A0E0C6ED30E0D6E020E0E6ED6
:10954800106A0D0E0F6E8EEC53F0496A250E486EA8
:1095580092EC32F00101FA93839012001A0E0D2456
:109568000F6E000E0E20106E0F28D96E000E102000
:10957800DA6EDF50126E116A1A0E0D24D96E000EC3
:109588000E20DA6EDF50111211C017F012C018F059
:10959800196A1A6A0BC0D9FF0CC0DAFF030EDE186D
:1095A80029E1140E0D240F6E000E0E20106E0F28E8
:1095B800D96E000E1020DA6EDF50126E116A140E8A
:1095C8000D24D96E000E0E20DA6EDF501110136EC6
:1095D8001250146E156A166A14C016F013C015F0EE
:1095E800146A136A135017121450181215501912CE
:1095F80016501A1217C00BF018C00CF019C00DF055
:109608001AC00EF01200226E2250D8A4040C20506A
:10961800211001E1040C54B0030C51B608D0090E16
:10962800D8901C361D361E361F36E82EF9D7215025
:1096380006E1020E205C03E2246A110E02D0246ABD
:10964800120E236E23C025F01CC014F01DC015F0A7
:109658001EC016F01FC017F02550C2EC54F00009C8
:109668001DE11AC00BF01BC00CF0020E0E6E0D6A45
:109678003AEC51F0000908E0020E1B262006D8A09B
:10968800210620502110EDE1120E251807E1146A79
:10969800156A166A176A0C0EC2EC54F01BEC57F0E8
:1096A80020502110D8A4010C000C155016100AE106
:1096B8007CC115F07DC116F01550161003E1156A2E
:1096C800166A120015C00FF016C010F017C011F07E
:1096D80018C012F028EC53F00F501526105016221F
:1096E80015C0D9FF16C0DAFFDF5006E101017C6B17
:1096F8007D6B156A166A120015C00FF016C010F0BF
:1097080017C011F018C012F04AEC53F00F5015248E
:1097180001017C6F105016207D6F7CC1D9FF7DC17F
:10972800DAFFDF5009E07CC1D9FF7DC1DAFF000E06
:10973800DF6A7C4B7D2B02D07C6B7D6B15C015F0EE
:1097480016C016F01200B96BBA6BACC0BBF0ADC056
:10975800BCF024D0B0C084F0B1C085F0B70E866FDD
:10976800876B896B010E886FBD0E8A6F8B6BFEEC61
:1097780011F0BD05BE1125E1B7C0BFF00D0EBF1930
:109788000DE0BBC0D9FFBCC0DAFFBFC0DFFFBB4BD9
:10979800BC2BB94BBA2B0A0EBF1913E0B269B369D7
:1097A800AEC0B4F0AFC0B5F0B251B427B351B523D1
:1097B800B451B95DBA51800AB66FB551800AB6592D
:1097C800C9E3BBC0D9FFBCC0DAFFDF6AB951BA111F
:1097D80003E1AC6BAD6B1200ACC0ACF0ADC0ADF04A
:1097E8001200436A20EE2AF03950D9263A50DA227C
:1097F8003B50DE1809E13C50DE1806E13D50DE180A
:1098080003E13E50DE1839E039C024F03AC025F0B3
:10981800C2EC40F0436E435030E12E0E39241A6EEC
:10982800000E3A201B6E3BC01CF03CC01DF03DC032
:109838001EF03EC01FF0216A010E206E20EE01F0DE
:109848003950D9263A50DA22DF5007EC4BF000099C
:1098580006E03B683C683D683E68010E436E20EEBA
:109868002AF03950D9263A50DA223BC0DEFF3CC0F4
:10987800DEFF3DC0DEFF3EC0DEFF43501200D4C015
:10988800DAF0D5C0DBF0DA0E0B6EBEEC43F00BC09D
:10989800DCF00CC0DDF00001DDBF0B0CD890DC352E
:1098A800D96EDD35DA6E8C0ED926010EDA22DECFBE
:1098B800D8F0DDCFD9F0D851D91105E0D8C0D9FFFB
:1098C800D9C0DAFFDF6AD251D31105E0D2C0D9FF7F
:1098D800D3C0DAFFDF6AD890DC35D96EDD35DA6EB1
:1098E8008C0ED926010EDA22D2C0DEFFD3C0DDFFEE
:1098F800D251D311D8B4000CD60501E0000CD20E19
:109908007C6F7D6BD40E7E6F7F6BAEEC00F0D76FF3
:10991800D751120003D00B4A0C2A0D2A0D50D96ECC
:10992800DA6ADF500E6E0BC0F6FF0CC0F7FF000EB0
:10993800F86E0E0EF76403D00800F55005D0F6CF88
:10994800E9FFF7CFEAFFEF500E1813E10BC0F6FF5F
:109958000CC0F7FF000EF86E0E0EF76403D0080077
:10996800F55005D0F6CFE9FFF7CFEAFFEF50000931
:10997800D2E10BC0F6FF0CC0F7FF000EF86E0E0E1A
:10998800F76403D00800F55005D0F6CFE9FFF7CF0C
:10999800EAFFEF500E6E0D50D96EDA6ADF500E5C9A
:1099A8000B6E0C6AD8A00C0612005050140D070E4E
:1099B800F324D96E010EF420DA6E000EDE24CD6F8A
:1099C800010EDE20CE6F000EDE20CF6F000EDE20EF
:1099D800D06F5050140D070EF324D96E010EF420E9
:1099E800DA6ECDC0DEFFCEC0DEFFCFC0DEFFD0C056
:1099F800DEFF5050140D070EF324D96E010EF4202B
:109A0800DA6EDECFD1F0DDCFD2F05050200D000E4F
:109A1800F324A66F020EF420A76FD1C0A8F0D2C01D
:109A2800A9F0AA6BAB6B14EC0FF0D36FD35103E022
:109A3800010E4E6E010C4E6A12000BC012F00CC0E3
:109A480013F00DC014F00EC015F00F06D8A01006C4
:109A58000F280CE110280AE10B6A0C6A1200124A5E
:109A6800132A144A152A0F06D8A0100612C0F6FFAA
:109A780013C0F7FF0800F55015E014C0D9FF15C052
:109A8800DAFFDF500FE00F5010100CE014C0D9FFC0
:109A980015C0DAFF12C0F6FF13C0F7FFDE50090049
:109AA800F518DDE012C0F6FF13C0F7FF0800F5CF88
:109AB80011F014C0D9FF15C0DAFFDF50115C0B6E2E
:109AC8000C6AD8A00C0612000CC012F00DC013F0DE
:109AD80012501310D8B4090C12C0D9FF13C0DAFF02
:109AE800DE50DE10D8B4090C12C0D9FF13C0DAFF5B
:109AF800DECF0EF0DDCF0FF00EC0D9FF0FC0DAFFBA
:109B0800DF50D8B4090C20EE02F01250D9261350B9
:109B1800DA2212C0E1FF13C0E2FF00EE06F0E650C1
:109B2800E926E550EA22DE50EE1813E1DE50EE1881
:109B3800D8A4090C12C0D9FF13C0DAFF10EE01F047
:109B4800DE50E126DD50E222E75011EC57F00E6EB0
:109B58000EB0090C000C24EE04F0DE50DE10FBE021
:109B680000C413F001C414F0060E1324D96E040EB9
:109B78001420DA6EDF50116E060E1324D96E060E0D
:109B88001420DA6EDF50126E134A142A0D68010E83
:109B98000E6E13C00FF014C010F00D500F160E50BB
:109BA80010160FC000F410C001F4F29E24EE04F069
:109BB800DE06000EDD5AF28E0BC0D9FF0CC0DAFFAC
:109BC80012C0DFFF24EE04F0010EDBBE05D0000E4C
:109BD800DE5C020EDE5801E28982115012000E503E
:109BE80002E00E5003E10C50CAEF56F00E50D96E49
:109BF800DA6A040ED926DE50DE1014E00E50D96E53
:109C0800DA6A040ED9260E50E16EE26A020EE126E7
:109C1800DE50E65CE650800A136EDE50800A135868
:109C2800D8B012000E50D96EDA6A020ED926DECFED
:109C38000FF0DDCF10F00E50D96EDA6ADECF11F0DA
:109C4800DDCF12F00F501124D96E10501220DA6EA9
:109C58000CC0DFFF0E50D96EDA6A020ED926DE2A52
:109C6800000EDD22000C0B500F02F3CF13F0F4CFDF
:109C780014F0156A166A0B501002F3501426F450AB
:109C88001522000E16220C500F02F3501426F45021
:109C98001522000E16220B501102F3501526F4500F
:109CA80016220C501002F3501526F45016220D50AF
:109CB8000F02F3501526F450162212500B02F350DF
:109CC80016260C501102F35016260D501002F350B0
:109CD80016260E500F02F350162613C00BF014C0B0
:109CE8000CF015C00DF016C00EF012000D0E606FCE
:109CF800FE0E616F88C162F089C163F0E0EC56F036
:109D080011D0030E0BD0050E4A6E0101886B896BCA
:109D18002DD00A0E03D0010E01D0020E4A6E26D0B5
:109D28004A6A24D088C148F089C149F0495009E0FD
:109D3800020A0DE00E0A0FE0010A11E02A0A13E0F8
:109D4800EFD748500A0ADDE01E0ADDE0E9D748509F
:109D5800BC0AE3E0E5D748501C0ADBE0E1D74850ED
:109D6800AC0AD9E0DDD748500F0ADAE14A501200B0
:109D7800150E116EC60EE82EFED7112EFCD700D098
:109D880020D0150E116EC60EE82EFED7112EFCD768
:109D980000D0010E0B6E0FC0F6FF10C0F7FF000ECB
:109DA800F86E0E0EF76403D00800F55005D0F6CF14
:109DB800E9FFF7CFEAFFEF5090EC52F00F4A102A74
:109DC800D7D70FC0F6FF10C0F7FF000EF86E0E0EC3
:109DD800F76403D00800F55005D0F6CFE9FFF7CFB8
:109DE800EAFFEF500009CDE11200136A146A156A00
:109DF800166A0F5010101110121029E0010E176E7C
:109E080006D0D8900F36103611361236172A12AEF1
:109E1800F8D7D89013361436153616360F500B5C13
:109E280010500C5811500D5812500E5809E30F508D
:109E38000B5E10500C5A11500D5A12500E5A1380C6
:109E4800D8901232113210320F32172EE2D713C0C7
:109E58000BF014C00CF015C00DF016C00EF0120077
:109E68000101956B4D6A866B876B020E946F839028
:109E7800936B926B506A030E506401D029D05050F6
:109E8800070D520EF324D96E010EF420DA6EDF6A44
:109E98005050070D510EF324D96E010EF420DA6EDE
:109EA800DF6A5050070D500EF324D96E010EF420CE
:109EB800DA6EDF6A5050070D530EF324D96E010E87
:109EC800F420DA6EDE6ADE6ADE6ADD6A502AD3D7EB
:109ED800506A1200136E0C0E131807E01BEC57F0B3
:109EE800B2EC56F0000901E1FF0C13504009F3EC05
:109EF80056F01050F3EC56F00F50F3EC56F00E50AD
:109F0800F3EC56F00D50F3EC56F0010E126E1350B0
:109F180002E1950E126E080E131802E1870E126EFA
:109F28001250F3EC56F00C0E131802E104EC57F043
:109F38000A0E126E04EC57F0116E11AE02D0122EFA
:109F4800F9D7115012000F501010D8B4000C0FC0E0
:109F5800D9FF10C0DAFFDF5001E1000C0FC00BF091
:109F680010C00CF0D0EC53F00BC011F00CC012F084
:109F7800020E1118121001E0000C130E0B6E0FC028
:109F8800D9FF10C0DAFFDF5067EC52F00009D8B4EF
:109F9800000C140E0B6E20EE01F00F50D926105055
:109FA800DA22DF5067EC52F0000901E1000C1338A7
:109FB800F00B14101200866A846A8B688968536AE9
:109FC800839283940101906B916B09D0000E9025C8
:109FD800D96E030E9121DA6EDF6A904B912B91BFF7
:109FE800F5D79105F3E3906B916B09D0340E90256A
:109FF800D96E0A0E9121DA6EDF6A904B912B91BFD0
:10A00800F5D79105F3E30F011769D6501F0B4009E7
:10A01800D66ED6980F0ED612D588D5120E01C29BD1
:10A02800D58E0F0C4EEC54F0CC0EA5EC56F0660E07
:10A03800A5EC56F088EC56F0156E155005E10F6A40
:10A04800106A116A126A1200136A146A1350150F03
:10A05800D96EDA6A88EC56F0DF6E134A142A14BEF9
:10A06800F5D7145003E1040E135CF0E318501710F1
:10A07800161003E1060E155CE2E315C00FF016C0DA
:10A0880010F017C011F018C012F01200506A030E39
:10A09800506401D029D05050070D520EF324D96EC8
:10A0A800010EF420DA6EDF6A5050070D510EF324CA
:10A0B800D96E010EF420DA6EDF6A5050070D500E8B
:10A0C800F324D96E010EF420DA6EDF6A5050070DC2
:10A0D800530EF324D96E010EF420DA6EDE6ADE6ABE
:10A0E800DE6ADD6A502AD3D7506A8390946B1200D7
:10A0F8000F5010101110121023E0010E136E06D02D
:10A10800D8900F36103611361236132A12AEF8D7F9
:10A118000F500B5C10500C5811500D5812500E581F
:10A1280008E30F500B5E10500C5A11500D5A125084
:10A138000E5AD8901232113210320F32132EE8D73D
:10A148000BC00BF00CC00CF00DC00DF00EC00EF0E3
:10A158001200196A1A6A536A186A21D078EC56F004
:10A168000B500C1011E0180E0B6E0C6AAFEC4DF092
:10A17800176E000E5324D96EDA6A030EDA2217C05E
:10A18800DFFF532A194A1A2A18AA07D0000E1924E1
:10A19800156E040E1A20166E12008EAC04D01ABE6C
:10A1A800DDD71A04DBE319C015F01AC016F0120047
:10A1B8000B6A0C6A5050140D070EF324D96E010E69
:10A1C800F420DA6EDE6ADE6ADE6ADD6A5050140D4B
:10A1D800130EF324D96E010EF420DA6EDF6A5050A4
:10A1E800140D0F0EF324D96E010EF420DA6EDE6A18
:10A1F800DE6ADE6ADD6A0B4A0C2A0CBEDBD70C501D
:10A2080003E1040E0B5CD6E383904E6A120089ECDE
:10A218003EF0CDC0E8F0CEC0E9F0E851E91105E024
:10A22800E8C0E4F0E9C0E5F012008FB414D0505053
:10A23800200D000EF324A66F020EF420A76F000E67
:10A24800A86F030EA96F010EAB6FAA6BE60EAC6F79
:10A25800A6EC0BF0EA6FEA5104E0EAC0E4F0E56B23
:10A268001200D9EC4CF0E46BE56B1200070E106E8F
:10A27800D00E0F6E0FD004EC57F0116E11280DE1BF
:10A28800E40E00D000D0E82EFCD700D000D00F0696
:10A29800D8A010060F501010EEE1FE0E111801E0C4
:10A2A800000C04EC57F00BC0D9FF0CC0DAFFDF6ECE
:10A2B8000B4A0C2A0D06D8A00E060D500E10F1E11F
:10A2C80004EC57F004EC57F0010C0BC012F00CC072
:10A2D80013F00DC014F00EC015F0166A176A0F06B9
:10A2E800D8A010060F2802E1102817E012C0D9FFE5
:10A2F80013C0DAFF124A132ADF50116E14C0D9FFB7
:10A3080015C0DAFF144A152ADF50115C166E176A59
:10A31800D8A0170616501710E2E016C00BF017C0A9
:10A328000CF012000BC011F00CC012F013D00F0685
:10A33800D8A010060DC0D9FF0EC0DAFF0D4A0E2AAC
:10A3480011C0E1FF12C0E2FF114A122ADFCFE7FF76
:10A35800E7500BE00F50101008E0E9D711C0D9FF03
:10A3680012C0DAFFDF6A114A122A0F06D8A01006B7
:10A378000F28F4E11028F2E11200F9EC54F000097A
:10A3880001E1000C0F50F3EC56F0FD0E0F181EE023
:10A39800020E116E106A0DC0D9FF0EC0DAFFDF5031
:10A3A800F3EC56F00D4A0E2A1006D8A011061050EC
:10A3B8001110F1E104EC57F004EC57F004EC57F0FD
:10A3C800126E12501F0B050A01E0000C010C15D08B
:10A3D8000CC0F6FF0DC0F7FF000EF86E0E0EF76406
:10A3E80003D00800F55005D0F6CFE9FFF7CFEAFF14
:10A3F800EF50D5EC56F00C4A0D2A0CC0F6FF0DC0F4
:10A40800F7FF000EF86E0E0EF76403D00800F55043
:10A4180005D0F6CFE9FFF7CFEAFFEF500009D8E102
:10A4280012000EC012F00FC013F010C014F011C0CB
:10A4380015F04EEC54F0CC0EA5EC56F0990EA5ECA8
:10A4480056F00C0EA5EC56F0166A176A1650120F45
:10A45800D96EDA6ADF50A5EC56F0164A172A17BEED
:10A46800F5D7175002E04EEF54F0040E165CEEE3F9
:10A478004EEF54F00001876FDD0E886FFA0E896F7A
:10A48800866B0AD088C0F6FF89C0F7FF884B892BF6
:10A498000800F550F7E1862B8751861907E088C038
:10A4A800F6FF89C0F7FF0800F550ECE1930E606FE6
:10A4B800FE0E616F87C062F0636B88C064F089C06C
:10A4C80065F0E0EF56F00C6E0B5001E1000C2F0E1A
:10A4D8000C6409D03A0E0C6006D00B50D96EDA6ABB
:10A4E8000C50D00F17D0400E0C6409D0470E0C60EA
:10A4F80006D00B50D96EDA6A0C50C90F0BD0600E1B
:10A508000C64000C670E0C60000C0B50D96EDA6AF4
:10A518000C50A90FDF6E010C0C6E87920A0EE82E04
:10A52800FED700D00BB002D0879401D08784000EEC
:10A538000E6E010E0D6E0CAE02D0838A01D0839A86
:10A54800D8900C36879000F000F0878000F000F07B
:10A5580087900D4A0E2A0EBEEED70E5003E1090E63
:10A568000D5CE9E38782120083800101FA832AEEF9
:10A5780034F092C1DFFF000EE8CF35FA0D0EE8CFB8
:10A5880036FA000EE8CF37FA8FA403D0600EE8CF72
:10A5980037FA8FA406D036CA4AF0200E4A124AC0AB
:10A5A80036FA496A040E486E92EC32F00101FA93C9
:10A5B800926B83901200010E0B6E0C6A888687825C
:10A5C800878400F000F0879400F000F00D6A0E6AAE
:10A5D8008DA602D00B500C12D8900B36879000F045
:10A5E80000F0878000F000F087900D4A0E2A0EBE1A
:10A5F800EFD70E5003E1030E0D5CEAE30C50120096
:10A60800838E83805050200D000EF3240001846F48
:10A61800020EF420856F340E866F0A0E876F010EC6
:10A62800896F886BAE0E8A6F8B6BFEEC11F001019F
:10A63800FA93AEC048F0AFC049F092EC32F0010195
:10A64800946B839E83901200136A146A04D00F4A95
:10A65800102A134A142A0FC0D9FF10C0DAFFDF509E
:10A6680010E011C00BF012C00CF00FC0D9FF10C0E1
:10A67800DAFFDF500D6E0E6A2EEC55F00B500C1001
:10A68800E6E113C00FF014C010F01200136A146A48
:10A6980004D00F4A102A134A142A0FC0D9FF10C039
:10A6A800DAFFDF5010E011C00BF012C00CF00FC041
:10A6B800D9FF10C0DAFFDF500D6E0E6A2EEC55F090
:10A6C8000B500C10E6E013C00FF014C010F012008D
:10A6D8009F0E136E146811C015F012C016F01350B7
:10A6E800152614501622165005E11A0E155C02E2C2
:10A6F800010E01D0000E176E186A1750181005E0E9
:10A708005F0E1114116E126A120011C011F012C0FE
:10A7180012F012000DC013F00EC014F00BC011F0AF
:10A728000CC012F010D013C0D9FF14C0DAFFDF50EC
:10A73800156E134A142A11C0D9FF12C0DAFF15C0CA
:10A74800DFFF114A122A0F06D8A010060F28EBE1E6
:10A758001028E9E1120020EE1AF00B50D9260C500F
:10A76800DA220DC0DFFF20EE1BF00B50D9260C506B
:10A77800DA220EC0DFFF20EE14F00B50D9260C5061
:10A78800DA220FC0DFFF20EE15F00B50D9260C504F
:10A79800DA221050DF6E12000BC00DF00CC00EF064
:10A7A80002D00B4A0C2A0BC0F6FF0CC0F7FF000EB4
:10A7B800F86E0E0EF76403D00800F55005D0F6CFFA
:10A7C800E9FFF7CFEAFFEF500009EBE10D500B5C12
:10A7D8000B6E0E500C580C6E12000007958101008C
:10A7E800400001000300005001F40101000007953A
:10A7F800810100400001000300005001F401010044
:10A8080000062305003E000000091127000006236A
:10A8180005003E000000091127000BC011F00CC014
:10A8280012F00DC013F00EC014F00ED013C0D9FFF3
:10A8380014C0DAFF11C0E1FF12C0E2FFDFCFE7FF6B
:10A84800134A142A114A122A0F06D8A010060F28F4
:10A85800EDE11028EBE112000B6E0B500EE022EC3C
:10A8680057F0200EE82EFED725EC57F0CC0E00D07E
:10A87800E82EFDD700D000D0120022EC57F0C00E11
:10A8880000D0E82EFDD725EC57F0350EE82EFED780
:10A8980000F0120022EC57F00A0E0C6EF80EE82EAB
:10A8A800FED70C2EFCD700D025EC57F0E00E00D0D8
:10A8B800E82EFDD7EAEC56F00D6E090E0C6E840EEC
:10A8C800E82EFED70C2EFCD725EC57F00D501200C1
:10A8D800730E776F6FC078F070C079F07A6B7B6B0E
:10A8E8007C6B7D6B780E696F71C06AF072C06BF01B
:10A8F800770E6C6F31EC20F000017A516F25D96E1C
:10A908007B517021DA6EDF6A000C000EF2BE010E78
:10A918000E6E0C50030B7F6E0BC07EFF0DC080FFC8
:10A928003F0E81168184F29E550E826EAA0E826EAB
:10A93800818281B2FED781940EB002D0F29E01D0FE
:10A94800F28E120002D00B4A0C2A0BC0F6FF0CC084
:10A95800F7FF0800F55009E00BC0F6FF0CC0F7FF41
:10A968000800F5500D180E10EEE10BC0F6FF0CC0F4
:10A97800F7FF0800F5500B6E0C6A1200186E18AE3F
:10A988000ED0189E0D6A0E6A0F6A106A370E6EECAA
:10A998004FF0196E010E196402D01950120014C03C
:10A9A8000DF015C00EF016C00FF017C010F01850BB
:10A9B8006EEF4FF0010E116E200E0B180C1011E007
:10A9C800F70E0D6E0E680BC00FF00CC010F00D5096
:10A9D8000F260E501022105003E1050E0F5C01E304
:10A9E800116A11C00BF00C6A1200130E0C6E880E5F
:10A9F8000B6E0ED004EC57F0FF0A0DE0E40E00D009
:10AA080000D0E82EFCD700D000D00B06D8A00C064A
:10AA18000B500C10EFE10B500C10D8A4010C000CDB
:10AA280048C046F049C047F001EC35F04A6E4A503C
:10AA38000FE148C00CF049C00DF068EC4DF04A6ECB
:10AA48004A5006E148C0D9FF49C0DAFFDE6ADD6A2C
:10AA58004A5012000BC0F6FF0CC0F7FF0800F55073
:10AA68000D1805E10BC00BF00CC00CF012000BC068
:10AA7800F6FF0CC0F7FF0B4A0C2A0800F550EAE174
:10AA88000B6A0C6A120060900F0E0F01596F070EC7
:10AA9800396F356F4F0E936E8A6A8A888A828A82E6
:10AAA800010E8F6E130E0E01B76F0F0EFA6F100E98
:10AAB800FC6F140EB86F140C9F0E0D6E0E68200EEE
:10AAC8000B100F6E000E0C10106E0D500F260E504E
:10AAD8001022105005E11A0E0F5C02E2010E01D09F
:10AAE800000E0B6E0C6A12009F869E84090E0E01E2
:10AAF800FD6F9F98890E9B6E9C6A9E989D8E9D887F
:10AB08009D9AC599F28AF28E9E909D9C9E9A9E8AE5
:10AB1800010198911200340E0B6E0A0E0C6E0E6A2B
:10AB28000D6A010E106E0F6A92EC42F02AEE34F0B4
:10AB380094C1DFFF496A010E486E92EC32F00101C0
:10AB4800946B1200340E0B6E0A0E0C6E0E6A0D6AB0
:10AB5800010E106E0F6A92EC42F0010EE8CF34FA43
:10AB68000101FA83496A486E92EC32F00101FA93C6
:10AB78001200186A196A09D017C00CF00D6A16C0BD
:10AB88000EF0F3EC4DF0184A192A18501424D96E17
:10AB980019501520DA6EDF50176E1750EDE11200CC
:10ABA8009F0E0D6E0E680BC00FF00CC010F00D500C
:10ABB8000F260E501022105005E11A0E0F5C02E20B
:10ABC800010E01D0000E0B6E0C6A1200BF0E0D6E46
:10ABD8000E680BC00FF00CC010F00D500F260E5071
:10ABE8001022105005E11A0E0F5C02E2010E01D08E
:10ABF800000E0B6E0C6A1200D00E0D6E0E680BC0A4
:10AC08000FF00CC010F00D500F260E5010221050EF
:10AC180005E10A0E0F5C02E2010E01D0000E0B6E78
:10AC28000C6A12000BC011F00CC012F008D011C051
:10AC3800D9FF12C0DAFF0DC0DFFF114A122A0F0632
:10AC4800D8A010060F28F3E11028F1E11200106ACD
:10AC5800110E0F6E09D00A0EE82EFED700D0010E95
:10AC68000B6E200E90EC52F00F06D8A010060F289D
:10AC7800F2E11028F0E112000B6E0B5009E0966A21
:10AC88004F0E936E220E966E400E956E968A400C6D
:10AC9800966A100E966E2A0E966E900E936EF4D7E4
:10ACA80022EC57F0200EE82EFED725EC57F0300E98
:10ACB800E82EFED7EAEC56F00C6EB00E00D0E82E67
:10ACC800FDD70C5012009150070B0B6E888A8DAA85
:10ACD80002D0080E0B26020E01019B1903E10B1C82
:10ACE8000F0B0B6E0B50120024EE04F0010EDBBEAE
:10ACF80005D0000EDE5C020EDE5801E2898204C433
:10AD08000BF005C40CF012000D6A0E6AD8900D32D3
:10AD180054EC56F0000901E00D8E0E2A070E0E6461
:10AD2800F5D70D501200000EE8CF00F4E8CF01F47B
:10AD3800E8CF02F4E8CF03F4E8CF04F4E8CF05F451
:10AD4800000C0C6E0D6A0C50010B30EC54F0D890CE
:10AD58000C320D2A070E0D64F6D7070C2AEC57F0B3
:10AD680004EC57F0F9EC54F0000901E0010C1BEC7D
:10AD780057F0000C0C50030B7F6E0BC07EFF3F0E8C
:10AD88008116818000F000F0805012000B6E03D015
:10AD98002CEC57F004000E01CDA9FAD70BC09AFF8E
:10ADA80012000B6E03D02CEC57F004000E01CDA955
:10ADB800FAD70BC09AFF1200620E476E60C018F0F7
:10ADC80061C019F0470E1A6E01EF28F088888DA827
:10ADD80003D0010E0B6E01D00B6A0B5012000B6EE4
:10ADE8000BC092FF95B0FED795A0FED792501200E7
:10ADF8000B6E02D0838C839C0B060B28FBE11200A0
:10AE0800926895B0FED795A0FED7925012001FE722
:10AE1800800103E800800103E8000B6E0B5001E09D
:10AE2800010C5450120083804E6A8390120028EC63
:10AE380057F004EF57F08390946B1200839888982A
:10AE4800120083988888120085801200859012006D
:03AE5800120001E4
:10FADC00004F4B004449534B5F455252004E4F541C
:10FAEC005F5245414459004E4F5F46494C45004ECC
:10FAFC004F545F4F50454E4544004E4F545F454E5A
:10FB0C0041424C4544004E4F5F46494C455F53596A
:10FB1C005354454D000020000D0A20253258202555
:10FB2C00325820253273202532732025327320253C
:10FB3C003273202532732025327320253273202511
:10FB4C0032732025347320253473202534732025FB
:10FB5C0034732025347320253473202534732025E9
:10FB6C00347320000D0A48504469736B204D6B2090
:10FB7C004949202831384634364B343029202573F6
:10FB8C00202573202573205374617274696E672E5F
:10FB9C002E2E0D0A000D0A547269656420746F20B4
:10FBAC0074616C6B207768696C7374206E6F742051
:10FBBC00616464726573736564000D0A4D6178202D
:10FBCC00566563746F72206469736B2025642025FD
:10FBDC006C642028256C582920000D0A25303258D9
:10FBEC00253032582053533830783A537461747539
:10FBFC00735B25645D20255820000D0A44736B73DC
:10FC0C00656C2069732025642C206E756D6265729D
:10FC1C002069732025642000466F756E6420616E28
:10FC2C00205254432066696C652061742025580D60
:10FC3C000A004C6F6F6B696E6720666F7220616E85
:10FC4C00205254432066696C650D0A0046696E6447
:10FC5C0046696C65206661696C65642073656172C8
:10FC6C0063680D0A000D0A5365656B20746F2025BF
:10FC7C006C64206661696C6564202564000D0A441F
:10FC8C0069736B2073656C656374206E756D62654A
:10FC9C0072202564005365656B696E6720746F2054
:10FCAC00736563746F722025580D0A0046696E6483
:10FCBC0046696C65206661696C6564207265616477
:10FCCC000D0A000D0A4F70656E696E6720657869C4
:10FCDC007374696E6720257320000D0A476F7420BA
:10FCEC00256C7520202D20726573657474696E67A0
:10FCFC00000D0A57616974696E6720666F72206324
:10FD0C0061726420000D0A46696C652025732069B8
:10FD1C0073206F70656E20000D0A57726F7465202A
:10FD2C006469736B6E6F3A202564000D0A4F706521
:10FD3C006E696E67206E657720257320000D0A258D
:10FD4C0030325825303258204578697420004E6F77
:10FD5C00742061204C4946206469736B0D0A000DB8
:10FD6C000A52656164206465736372696265200080
:10FD7C000D0A46696C65202558206973202573206F
:10FD8C00000D0A4469736B20255820697320257374
:10FD9C0020000D0A48737420627974657332202533
:10FDAC0064000D0A5772697465206661696C2025C0
:10FDBC0064000D0A52656164696E67205254430DEC
:10FDCC000A000D0A416D69676F2039313231440DDB
:10FDDC000A000D0A44736B73656C206973202564EB
:10FDEC0020000D0A526561642025642062797465D7
:10FDFC007300566563746F722069732025580D0A61
:10FE0C00000D0A5353383065786563202564200053
:10FE1C00222A2B2C3A3B3C3D3E3F5B5D7C7F000D08
:10FE2C000A4F70656E696E672025732020000D0ADD
:10FE3C00446562756720697320256420000D0A50A3
:10FE4C00726F746F20697320256420000D0A52654F
:10FE5C00616420636F6E66696720000D0A46696CE9
:10FE6C00656E616D6520257320002041544E206124
:10FE7C007373657274656420000D0A466F726D6150
:10FE8C007474696E67200072633D25752046525F5D
:10FE9C0025730D0A002A2A20566572696679202A74
:10FEAC002A000D0A73627974657331202564000D84
:10FEBC000A4E6F206361726420256400646573636D
:10FECC00726962652E636667002F6C696664617483
:10FEDC00612E62696E000D0A257320255820255865
:10FEEC000D0A000D0A4D6F756E74696E6720004E19
:10FEFC006F762033302032303230004C6F616469C1
:10FF0C006E672E2E2E0068706469736B2E636667A5
:10FF1C0000466D74206578697420005B5352512043
:10FF2C006F66665D0030393A35303A3132005B2508
:10FF3C0032582025645D005B535251206F6E5D007A
:10FF4C0048504469736B20004E6F206361726400EB
:10FF5C002D3E202558200072633D2564200044531B
:10FF6C004B53454C004E414D452558004449534B8D
:10FF7C002558005B4D4C415D0044454255470050AF
:10FF8C00524F544F0052656164790020253032582D
:10FF9C00007B4552527D00302E31350049464320BE
:10FFAC0000454F49200052454E200041544E200040
:10FFBC00535251200044415620004E444143004EC0
:10FFCC005246440052544300434C4B0020255800E9
:10FFDC0025325800207C200044300044310044324B
:10FFEC0000443300443400443500443600443700A8
:04FFFC002563000079
:020000040020DA
:10000000FF0FFF0FFF0FFF0FFF0FFF0FFF0FFF0F80
:020000040030CA
:0C0000008CFFFFFF8EFFFFFFFFFFFFFFE4
:00000001FF
